:020000040000FA
:3C000000FFFF627515FFFFFFFFFFFFFFFFFFFFFFFFFFFFFFFFFFFFFFFFFFFFFFFFFFFFFFFFFFFFFFFFFFFFFFFFFFFFFFFFFFFFFFFFFFFFFFFFFFFFFFFFFFFFFF11
:3C003C00000000000000000000000000000000000000000000000000000000000000000000000000000000000000000000000000000000000000000000001EFE6C
:3C007800000000000000000000000000000000000000000000000000000000000000000000000000000000000000000000000000000000000000000000001EFE30
:3C00B4000000000000000000000004800000000000000000000000000000000000000000000004000400000000000000000000000080040000000000000092FE70
:3C00F000000004800480048004800480048004800480048004800480048004800480048004800480048004800480048004800480048004800480048000001EFECC
:3C012C00000004800480048004800480048004800480048004800480048004800480048004800480048004800480048004800480048004800480048000001EFE8F
:3C016800000004000480000000000480000000000480040004800080040004000000000000000400048004000480008004000480008004800400048000001AFEFF
:3C01A4000000008000000480048004800480048000000080000004000080008004800480048004800400008000000400008000000480040000800000000096FED3
:3C01E0000000008000000480048004800480048000000080000004000080008004800480048004800400008000000400008000000480040000800000000096FE97
:3C021C00000000000000000000000000000000000000000000000000000000000000000000000000000000000000000000000000000000000000000000001EFE8A
:3C025800000000000000000000000000000000000000000000000000000000000000000000000000000000000000000000000000000000000000000000001EFE4E
:3C029400000000000000000000000000000000000000000000000000000000000000000000000000000000000000000000000000000000000000000000001EFE12
:3C02D000020000000000000000000000000000000000000000000000000000000000000000000000000000000000000000000000000000000000000000002FFFC2
:3C030C00020000000000000000000000000000000000000000000000000000000000000000000000000000000000000000000000000000000000000000002FFF85
:3C034800020000000000000000000000000000000000000000000000000000000000000000000000000000000000000000000000000000000000000000002FFF49
:3C038400000000000000000000000000000000000000000000000000000000000000000000000000000000000000000000000000000000000000000000001EFE21
:3C03C000000000000000000000000000000000000000000000000000000000000000000000000000000000000000000000000000000000000000000000001EFEE5
:3C03FC00000000000000000000000000000000000000000000000000000000000000000000000000000000000000000000000000000000000000000000001EFEA9
:3C043800000000000000000000000000000000000000000000000000000000000000000000000000000000000000000000000000000000000000000000001EFE6C
:3C047400000000000000000000000000000000000000000000000000000000000000000000000000000000000000000000000000000000000000000000001EFE30
:3C04B000020000000000000000000000000000000000000000000000000000000000000000000000000000000000000000000000000000000000000000002FFFE0
:3C04EC00020000000000000000000000000000000000000000000000000000000000000000000000000000000000000000000000000000000000000000002FFFA4
:3C052800000000000000000000000000000000000000000000000000000000000000000000000000000000000000000000000000000000000000000000001EFE7B
:3C056400020000000000000000000000000000000000000000000000000000000000000000000000000000000000000000000000000000000000000000002FFF2B
:3C05A000020000000000000000000000000000000000000000000000000000000000000000000000000000000000000000000000000000000000000000002FFFEF
:3C05DC00000000000000000000000000000000000000000000000000000000000000000000000000000000000000000000000000000000000000000000001EFEC7
:3C061800000000000000000000000000000000000000000000000000000000000000000000000000000000000000000000000000000000000000000000001EFE8A
:3C065400000000000000000000000000000000000000000000000000000000000000000000000000000000000000000000000000000000000000000000001EFE4E
:3C069000020000000000000000000000000000000000000000000000000000000000000000000000000000000000000000000000000000000000000000002FFFFE
:3C06CC00020000000000000000000000000000000000000000000000000000000000000000000000000000000000000000000000000000000000000000002FFFC2
:3C070800020000000000000000000000000000000000000000000000000000000000000000000000000000000000000000000000000000000000000000002FFF85
:3C074400000000000000000000000000000000000000000000000000000000000000000000000000000000000000000000000000000000000000000000001EFE5D
:3C078000000000000000000000000000000000000000000000000000000000000000000000000000000000000000000000000000000000000000000000001EFE21
:3C07BC00000000000000000000000000000000000000000000000000000000000000000000000000000000000000000000000000000000000000000000001EFEE5
:3C07F800000000000000000000000000000000000000000000000000000000000000000000000000000000000000000000000000000000000000000000001EFEA9
:3C083400000000000000000000000000000000000000000000000000000000000000000000000000000000000000000000000000000000000000000000001EFE6C
:3C087000020000000000000000000000000000000000000000000000000000000000000000000000000000000000000000000000000000000000000000002FFF1C
:3C08AC00020000000000000000000000000000000000000000000000000000000000000000000000000000000000000000000000000000000000000000002FFFE0
:3C08E800020000000000000000000000000000000000000000000000000000000000000000000000000000000000000000000000000000000000000000002FFFA4
:3C092400000000000000000000000000000000000000000000000000000000000000000000000000000000000000000000000000000000000000000000001EFE7B
:3C096000000000000000000000000000000000000000000000000000000000000000000000000000000000000000000000000000000000000000000000001EFE3F
:3C099C00000000000000000000000000000000000000000000000000000000000000000000000000000000000000000000000000000000000000000000001EFE03
:3C09D800000000000000000000000000000000000000000000000000000000000000000000000000000000000000000000000000000000000000000000001EFEC7
:3C0A1400000000000000000000000000000000000000000000000000000000000000000000000000000000000000000000000000000000000000000000001EFE8A
:3C0A5000020000000000000000000000000000000000000000000000000000000000000000000000000000000000000000000000000000000000000000002FFF3A
:3C0A8C00020000000000000000000000000000000000000000000000000000000000000000000000000000000000000000000000000000000000000000002FFFFE
:3C0AC800020000000000000000000000000000000000000000000000000000000000000000000000000000000000000000000000000000000000000000002FFFC2
:3C0B0400000000000000000000000000000000000000000000000000000000000000000000000000000000000000000000000000000000000000000000001EFE99
:3C0B4000000000000000000000000000000000000000000000000000000000000000000000000000000000000000000000000000000000000000000000001EFE5D
:3C0B7C00000000000000000000000000000000000000000000000000000000000000000000000000000000000000000000000000000000000000000000001EFE21
:3C0BB800000000000000000000000000000000000000000000000000000000000000000000000000000000000000000000000000000000000000000000001EFEE5
:3C0BF400000000000000000000000000000000000000000000000000000000000000000000000000000000000000000000000000000000000000000000001EFEA9
:3C0C3000020000000000000000000000000000000000000000000000000000000000000000000000000000000000000000000000000000000000000000002FFF58
:3C0C6C00020000000000000000000000000000000000000000000000000000000000000000000000000000000000000000000000000000000000000000002FFF1C
:3C0CA800020000000000000000000000000000000000000000000000000000000000000000000000000000000000000000000000000000000000000000003EFED2
:3C0CE400000000000000000000000000000000000000000000000000000000000000000000000000000000000000000000000000000000000000000000000FFFC6
:3C0D2000000000000000000000000000000000000000000000000000000000000000000000000000000000000000000000000000000000000000000000000FFF89
:3C0D5C00000000000000000000000000000000000000000000000000000000000000000000000000000000000000000000000000000000000000000000001EFE3F
:3C0D9800000000000000000000000000000000000000000000000000000000000000000000000000000000000000000000000000000000000000000000001EFE03
:3C0DD400000000000000000000000000000000000000000000000000000000000000000000000000000000000000000000000000000000000000000000001EFEC7
:3C0E1000020000000000000000000000000000000000000000000000000000000000000000000000000000000000000000000000000000000000000000002FFF76
:3C0E4C00020000000000000000000000000000000000000000000000000000000000000000000000000000000000000000000000000000000000000000002FFF3A
:3C0E8800000000000000000000000000000000000000000000000000000000000000000000000000000000000000000000000000000000000000000000001EFE12
:3C0EC400020000000000000000000000000000000000000000000000000000000000000000000000000000000000000000000000000000000000000000002FFFC2
:3C0F0000020000000000000000000000000000000000000000000000000000000000000000000000000000000000000000000000000000000000000000002FFF85
:3C0F3C00000000000000000000000000000000000000000000000000000000000000000000000000000000000000000000000000000000000000000000001EFE5D
:3C0F7800000000000000000000000000000000000000000000000000000000000000000000000000000000000000000000000000000000000000000000001EFE21
:3C0FB400000000000000000000000000000000000000000000000000000000000000000000000000000000000000000000000000000000000000000000001EFEE5
:3C0FF000020000000000000000000000000000000000000000000000000000000000000000000000000000000000000000000000000000000000000000002FFF95
:3C102C00020000000000000000000000000000000000000000000000000000000000000000000000000000000000000000000000000000000000000000002FFF58
:3C106800000000000000000000000000000000000000000000000000000000000000000000000000000000000000000000000000000000000000000000001EFE30
:3C10A400020000000000000000000000000000000000000000000000000000000000000000000000000000000000000000000000000000000000000000002FFFE0
:3C10E000020000000000000000000000000000000000000000000000000000000000000000000000000000000000000000000000000000000000000000002FFFA4
:3C111C00000000000000000000000000000000000000000000000000000000000000000000000000000000000000000000000000000000000000000000001EFE7B
:3C115800000000000000000000000000000000000000000000000000000000000000000000000000000000000000000000000000000000000000000000001EFE3F
:3C119400000000000000000000000000000000000000000000000000000000000000000000000000000000000000000000000000000000000000000000001EFE03
:3C11D000020000000000000000000000000000000000000000000000000000000000000000000000000000000000000000000000000000000000000000002FFFB3
:3C120C00020000000000000000000000000000000000000000000000000000000000000000000000000000000000000000000000000000000000000000002FFF76
:3C124800000000000000000000000000000000000000000000000000000000000000000000000000000000000000000000000000000000000000000000001EFE4E
:3C128400020000000000000000000000000000000000000000000000000000000000000000000000000000000000000000000000000000000000000000002FFFFE
:3C12C000020000000000000000000000000000000000000000000000000000000000000000000000000000000000000000000000000000000000000000002FFFC2
:3C12FC00000000000000000000000000000000000000000000000000000000000000000000000000000000000000000000000000000000000000000000001EFE9A
:3C133800000000000000000000000000000000000000000000000000000000000000000000000000000000000000000000000000000000000000000000001EFE5D
:3C137400000000000000000000000000000000000000000000000000000000000000000000000000000000000000000000000000000000000000000000001EFE21
:3C13B000020000000000000000000000000000000000000000000000000000000000000000000000000000000000000000000000000000000000000000002FFFD1
:3C13EC00020000000000000000000000000000000000000000000000000000000000000000000000000000000000000000000000000000000000000000002FFF95
:3C142800008000800080008000800080008000800080008000800080008000800080008000800080008000800080008000800080008000800080008000009EFEEC
:3C146400020000000000000000000000000000000000000000000000000000000000000000000000000000000000000000000000000000000000000000002FFF1C
:3C14A000020000000000000000000000000000000000000000000000000000000000000000000000000000000000000000000000000000000000000000002FFFE0
:3C14DC00000000000000000000000000000000000000000000000000000000000000000000000000000000000000000000000000000000000000000000001EFEB8
:3C151800000000000000000000000000000000000000000000000000000000000000000000000000000000000000000000000000000000000000000000001EFE7B
:3C155400000000000000000000000000000000000000000000000000000000000000000000000000000000000000000000000000000000000000000000001EFE3F
:3C159000000000000000000000000000000000000000000000000000000000000000000000000000000000000000000000000000000000000000000000001EFE03
:3C15CC00000000000000000000000000000000000000000000000000000000000000000000000000000000000000000000000000000000000000000000001EFEC7
:3C160800000000000000000000000000000000000000000000000000000000000000000000000000000000000000000000000000000000000000000000001EFE8A
:3C164400000000000000000000000000000000000000000000000000000000000000000000000000000000000000000000000000000000000000000000001EFE4E
:3C168000000000000000000000000000000000000000000000000000000000000000000000000000000000000000000000000000000000000000000000001EFE12
:3C16BC00000000000000000000000000000000000000000000000000000000000000000000000000000000000000000000000000000000000000000000001EFED6
:3C16F800000000000000000000000000000000000000000000000000000000000000000000000000000000000000000000000000000000000000000000001EFE9A
:3C173400000000000000000000000000000000000000000000000000000000000000000000000000000000000000000000000000000000000000000000001EFE5D
:3C177000000000000000000000000000000000000000000000000000000000000000000000000000000000000000000000000000000000000000000000001EFE21
:3C17AC00000000000000000000000000000000000000000000000000000000000000000000000000000000000000000000000000000000000000000000001EFEE5
:3C17E800000000000000000000000000000000000000000000000000000000000000000000000000000000000000000000000000000000000000000000001EFEA9
:3C182400000000000000000000000000000000000000000000000000000000000000000000000000000000000000000000000000000000000000000000001EFE6C
:3C186000000000000000000000000000000000000000000000000000000000000000000000000000000000000000000000000000000000000000000000001EFE30
:3C189C00000000000000000000000000000000000000000000000000000000000000000000000000000000000000000000000000000000000000000000001EFEF4
:3C18D800000000000000000000000000000000000000000000000000000000000000000000000000000000000000000000000000000000000000000000001EFEB8
:3C191400000000000000000000000000000000000000000000000000000000000000000000000000000000000000000000000000000000000000000000001EFE7B
:3C195000000000000000000000000000000000000000000000000000000000000000000000000000000000000000000000000000000000000000000000001EFE3F
:3C198C00000000000000000000000000000000000000000000000000000000000000000000000000000000000000000000000000000000000000000000001EFE03
:3C19C800000000000000000000000000000000000000000000000000000000000000000000000000000000000000000000000000000000000000000000001EFEC7
:3C1A0400000000000000000000000000000000000000000000000000000000000000000000000000000000000000000000000000000000000000000000001EFE8A
:3C1A4000000000000000000000000000000000000000000000000000000000000000000000000000000000000000000000000000000000000000000000001EFE4E
:3C1A7C00000000000000000000000000000000000000000000000000000000000000000000000000000000000000000000000000000000000000000000001EFE12
:3C1AB800000000000000000000000000000000000000000000000000000000000000000000000000000000000000000000000000000000000000000000001EFED6
:3C1AF400000000000000000000000000000000000000000000000000000000000000000000000000000000000000000000000000000000000000000000001EFE9A
:3C1B3000000000000000000000000000000000000000000000000000000000000000000000000000000000000000000000000000000000000000000000001EFE5D
:3C1B6C00000000000000000000000000000000000000000000000000000000000000000000000000000000000000000000000000000000000000000000001EFE21
:3C1BA800000000000000000000000000000000000000000000000000000000000000000000000000000000000000000000000000000000000000000000001EFEE5
:3C1BE400000000000000000000000000000000000000000000000000000000000000000000000000000000000000000000000000000000000000000000001EFEA9
:3C1C2000000000000000000000000000000000000000000000000000000000000000000000000000000000000000000000000000000000000000000000001EFE6C
:3C1C5C00000000000000000000000000000000000000000000000000000000000000000000000000000000000000000000000000000000000000000000001EFE30
:3C1C9800000000000000000000000000000000000000000000000000000000000000000000000000000000000000000000000000000000000000000000001EFEF4
:3C1CD400000000000000000000000000000000000000000000000000000000000000000000000000000000000000000000000000000000000000000000001EFEB8
:3C1D1000000000000000000000000000000000000000000000000000000000000000000000000000000000000000000000000000000000000000000000001EFE7B
:3C1D4C00000000000000000000000000000000000000000000000000000000000000000000000000000000000000000000000000000000000000000000000FFF4D
:3C1D8800000000000000000000000000000000000000000000000000000000000000000000000000000000000000000000000000000000000000000000001EFE03
:3C1DC400000000000000000000000000000000000000000000000000000000000000000000000000000000000000000000000000000000000000000000001EFEC7
:3C1E0000020000000000000000000000000000000000000000000000000000000000000000000000000000000000000000000000000000000000000000003EFE68
:3C1E3C00020000000000000000000000000000000000000000000000000000000000000000000000000000000000000000000000000000000000000000002FFF3A
:3C1E7800000000000000000000000000000000000000000000000000000000000000000000000000000000000000000000000000000000000000000000000FFF20
:3C1EB400020000000000000000000000000000000000000000000000000000000000000000000000000000000000000000000000000000000000000000003EFEB4
:3C1EF000020000000000000000000000000000000000000000000000000000000000000000000000000000000000000000000000000000000000000000003EFE78
:3C1F2C00020000000000000000000000000000000000000000000000000000000000000000000000000000000000000000000000000000000000000000003EFE3B
:3C1F6800000000000000000000000000000000000000000000000000000000000000000000000000000000000000000000000000000000000000000000001EFE21
:3C1FA400000000000000000000000000000000000000000000000000000000000000000000000000000000000000000000000000000000000000000000001EFEE5
:3C1FE000020000000000000000000000000000000000000000000000000000000000000000000000000000000000000000000000000000000000000000002FFF95
:3C201C00020000000000000000000000000000000000000000000000000000000000000000000000000000000000000000000000000000000000000000002FFF58
:3C205800020000000000000000000000000000000000000000000000000000000000000000000000000000000000000000000000000000000000000000002FFF1C
:3C209400020000000000000000000000000000000000000000000000000000000000000000000000000000000000000000000000000000000000000000003EFED2
:3C20D000020000000000000000000000000000000000000000000000000000000000000000000000000000000000000000000000000000000000000000003EFE96
:3C210C00000000000000000000000000000000000000000000000000000000000000000000000000000000000000000000000000000000000000000000001EFE7B
:3C214800000000000000000000000000000000000000000000000000000000000000000000000000000000000000000000000000000000000000000000001EFE3F
:3C218400000000000000000000000000000000000000000000000000000000000000000000000000000000000000000000000000000000000000000000001EFE03
:3C21C000020000000000000000000000000000000000000000000000000000000000000000000000000000000000000000000000000000000000000000002FFFB3
:3C21FC00020000000000000000000000000000000000000000000000000000000000000000000000000000000000000000000000000000000000000000002FFF77
:3C223800000000000000000000000000000000000000000000000000000000000000000000000000000000000000000000000000000000000000000000001EFE4E
:3C227400020000000000000000000000000000000000000000000000000000000000000000000000000000000000000000000000000000000000000000002FFFFE
:3C22B000020000000000000000000000000000000000000000000000000000000000000000000000000000000000000000000000000000000000000000002FFFC2
:3C22EC00020000000000000000000000000000000000000000000000000000000000000000000000000000000000000000000000000000000000000000003EFE78
:3C232800000000000000000000000000000000000000000000000000000000000000000000000000000000000000000000000000000000000000000000001EFE5D
:3C236400000000000000000000000000000000000000000000000000000000000000000000000000000000000000000000000000000000000000000000001EFE21
:3C23A000020000000000000000000000000000000000000000000000000000000000000000000000000000000000000000000000000000000000000000002FFFD1
:3C23DC00020000000000000000000000000000000000000000000000000000000000000000000000000000000000000000000000000000000000000000002FFF95
:3C241800020000000000000000000000000000000000000000000000000000000000000000000000000000000000000000000000000000000000000000003EFE4A
:3C245400020000000000000000000000000000000000000000000000000000000000000000000000000000000000000000000000000000000000000000002FFF1C
:3C249000020000000000000000000000000000000000000000000000000000000000000000000000000000000000000000000000000000000000000000002FFFE0
:3C24CC00000000000000000000000000000000000000000000000000000000000000000000000000000000000000000000000000000000000000000000000FFFC6
:3C250800000000000000000000000000000000000000000000000000000000000000000000000000000000000000000000000000000000000000000000001EFE7B
:3C254400000000000000000000000000000000000000000000000000000000000000000000000000000000000000000000000000000000000000000000001EFE3F
:3C258000020000000000000000000000000000000000000000000000000000000000000000000000000000000000000000000000000000000000000000003EFEE1
:3C25BC00020000000000000000000000000000000000000000000000000000000000000000000000000000000000000000000000000000000000000000002FFFB3
:3C25F800000000000000000000000000000000000000000000000000000000000000000000000000000000000000000000000000000000000000000000000FFF99
:3C263400020000000000000000000000000000000000000000000000000000000000000000000000000000000000000000000000000000000000000000003EFE2C
:3C267000020000000000000000000000000000000000000000000000000000000000000000000000000000000000000000000000000000000000000000003EFEF0
:3C26AC00000000000000000000000000000000000000000000000000000000000000000000000000000000000000000000000000000000000000000000001EFED6
:3C26E800000000000000000000000000000000000000000000000000000000000000000000000000000000000000000000000000000000000000000000001EFE9A
:3C272400000000000000000000000000000000000000000000000000000000000000000000000000000000000000000000000000000000000000000000001EFE5D
:3C276000020000000000000000000000000000000000000000000000000000000000000000000000000000000000000000000000000000000000000000002FFF0D
:3C279C00020000000000000000000000000000000000000000000000000000000000000000000000000000000000000000000000000000000000000000002FFFD1
:3C27D800000000000000000000000000000000000000000000000000000000000000000000000000000000000000000000000000000000000000000000001EFEA9
:3C281400020000000000000000000000000000000000000000000000000000000000000000000000000000000000000000000000000000000000000000002FFF58
:3C285000020000000000000000000000000000000000000000000000000000000000000000000000000000000000000000000000000000000000000000002FFF1C
:3C288C00000000000000000000000000000000000000000000000000000000000000000000000000000000000000000000000000000000000000000000000FFF02
:3C28C800000000000000000000000000000000000000000000000000000000000000000000000000000000000000000000000000000000000000000000001EFEB8
:3C290400000000000000000000000000000000000000000000000000000000000000000000000000000000000000000000000000000000000000000000001EFE7B
:3C294000020000000000000000000000000000000000000000000000000000000000000000000000000000000000000000000000000000000000000000003EFE1D
:3C297C00020000000000000000000000000000000000000000000000000000000000000000000000000000000000000000000000000000000000000000002FFFEF
:3C29B800000000000000000000000000000000000000000000000000000000000000000000000000000000000000000000000000000000000000000000000FFFD5
:3C29F400020000000000000000000000000000000000000000000000000000000000000000000000000000000000000000000000000000000000000000003EFE69
:3C2A3000020000000000000000000000000000000000000000000000000000000000000000000000000000000000000000000000000000000000000000003EFE2C
:3C2A6C00000000000000000000000000000000000000000000000000000000000000000000000000000000000000000000000000000000000000000000000FFF20
:3C2AA800000000000000000000000000000000000000000000000000000000000000000000000000000000000000000000000000000000000000000000001EFED6
:3C2AE400000000000000000000000000000000000000000000000000000000000000000000000000000000000000000000000000000000000000000000001EFE9A
:3C2B2000020000000000000000000000000000000000000000000000000000000000000000000000000000000000000000000000000000000000000000003EFE3B
:3C2B5C00020000000000000000000000000000000000000000000000000000000000000000000000000000000000000000000000000000000000000000002FFF0D
:3C2B9800000000000000000000000000000000000000000000000000000000000000000000000000000000000000000000000000000000000000000000000FFFF3
:3C2BD400020000000000000000000000000000000000000000000000000000000000000000000000000000000000000000000000000000000000000000003EFE87
:3C2C1000020000000000000000000000000000000000000000000000000000000000000000000000000000000000000000000000000000000000000000003EFE4A
:3C2C4C00000000000000000000000000000000000000000000000000000000000000000000000000000000000000000000000000000000000000000000001EFE30
:3C2C8800000000000000000000000000000000000000000000000000000000000000000000000000000000000000000000000000000000000000000000001EFEF4
:3C2CC400000000000000000000000000000000000000000000000000000000000000000000000000000000000000000000000000000000000000000000001EFEB8
:3C2D0000020000000000000000000000000000000000000000000000000000000000000000000000000000000000000000000000000000000000000000002FFF67
:3C2D3C00020000000000000000000000000000000000000000000000000000000000000000000000000000000000000000000000000000000000000000002FFF2B
:3C2D7800020000000000000000000000000000000000000000000000000000000000000000000000000000000000000000000000000000000000000000003EFEE1
:3C2DB400000000000000000000000000000000000000000000000000000000000000000000000000000000000000000000000000000000000000000000000FFFD5
:3C2DF000000000000000000000000000000000000000000000000000000000000000000000000000000000000000000000000000000000000000000000000FFF99
:3C2E2C00000000000000000000000000000000000000000000000000000000000000000000000000000000000000000000000000000000000000000000000FFF5C
:3C2E6800000000000000000000000000000000000000000000000000000000000000000000000000000000000000000000000000000000000000000000001EFE12
:3C2EA400000000000000000000000000000000000000000000000000000000000000000000000000000000000000000000000000000000000000000000001EFED6
:3C2EE000020000000000000000000000000000000000000000000000000000000000000000000000000000000000000000000000000000000000000000003EFE78
:3C2F1C00020000000000000000000000000000000000000000000000000000000000000000000000000000000000000000000000000000000000000000002FFF49
:3C2F5800008000800080008000800080008000800080008000800080008000800080008000800080008000800080008000800080008000800080008000008FFFAF
:3C2F9400020000000000000000000000000000000000000000000000000000000000000000000000000000000000000000000000000000000000000000003EFEC3
:3C2FD000020000000000000000000000000000000000000000000000000000000000000000000000000000000000000000000000000000000000000000003EFE87
:3C300C00000000000000000000000000000000000000000000000000000000000000000000000000000000000000000000000000000000000000000000001EFE6C
:3C304800000000000000000000000000000000000000000000000000000000000000000000000000000000000000000000000000000000000000000000001EFE30
:3C308400000000000000000000000000000000000000000000000000000000000000000000000000000000000000000000000000000000000000000000001EFEF4
:3C30C000000000000000000000000000000000000000000000000000000000000000000000000000000000000000000000000000000000000000000000001EFEB8
:3C30FC00000000000000000000000000000000000000000000000000000000000000000000000000000000000000000000000000000000000000000000001EFE7C
:3C313800000000000000000000000000000000000000000000000000000000000000000000000000000000000000000000000000000000000000000000001EFE3F
:3C317400000000000000000000000000000000000000000000000000000000000000000000000000000000000000000000000000000000000000000000001EFE03
:3C31B000000000000000000000000000000000000000000000000000000000000000000000000000000000000000000000000000000000000000000000001EFEC7
:3C31EC00000000000000000000000000000000000000000000000000000000000000000000000000000000000000000000000000000000000000000000001EFE8B
:3C322800000000000000000000000000000000000000000000000000000000000000000000000000000000000000000000000000000000000000000000001EFE4E
:3C326400000000000000000000000000000000000000000000000000000000000000000000000000000000000000000000000000000000000000000000001EFE12
:3C32A000000000000000000000000000000000000000000000000000000000000000000000000000000000000000000000000000000000000000000000001EFED6
:3C32DC00000000000000000000000000000000000000000000000000000000000000000000000000000000000000000000000000000000000000000000001EFE9A
:3C331800000000000000000000000000000000000000000000000000000000000000000000000000000000000000000000000000000000000000000000001EFE5D
:3C335400000000000000000000000000000000000000000000000000000000000000000000000000000000000000000000000000000000000000000000001EFE21
:3C339000000000000000000000000000000000000000000000000000000000000000000000000000000000000000000000000000000000000000000000001EFEE5
:3C33CC00000000000000000000000000000000000000000000000000000000000000000000000000000000000000000000000000000000000000000000001EFEA9
:3C340800000000000000000000000000000000000000000000000000000000000000000000000000000000000000000000000000000000000000000000001EFE6C
:3C344400000000000000000000000000000000000000000000000000000000000000000000000000000000000000000000000000000000000000000000001EFE30
:3C348000000000000000000000000000000000000000000000000000000000000000000000000000000000000000000000000000000000000000000000001EFEF4
:3C34BC00000000000000000000000000000000000000000000000000000000000000000000000000000000000000000000000000000000000000000000001EFEB8
:3C34F800000000000000000000000000000000000000000000000000000000000000000000000000000000000000000000000000000000000000000000001EFE7C
:3C353400000000000000000000000000000000000000000000000000000000000000000000000000000000000000000000000000000000000000000000001EFE3F
:3C357000000000000000000000000000000000000000000000000000000000000000000000000000000000000000000000000000000000000000000000001EFE03
:3C35AC00000000000000000000000000000000000000000000000000000000000000000000000000000000000000000000000000000000000000000000001EFEC7
:3C35E800000000000000000000000000000000000000000000000000000000000000000000000000000000000000000000000000000000000000000000001EFE8B
:3C362400000000000000000000000000000000000000000000000000000000000000000000000000000000000000000000000000000000000000000000001EFE4E
:3C366000000000000000000000000000000000000000000000000000000000000000000000000000000000000000000000000000000000000000000000001EFE12
:3C369C00000000000000000000000000000000000000000000000000000000000000000000000000000000000000000000000000000000000000000000001EFED6
:3C36D800000000000000000000000000000000000000000000000000000000000000000000000000000000000000000000000000000000000000000000001EFE9A
:3C371400000000000000000000000000000000000000000000000000000000000000000000000000000000000000000000000000000000000000000000001EFE5D
:3C375000000000000000000000000000000000000000000000000000000000000000000000000000000000000000000000000000000000000000000000001EFE21
:3C378C00000000000000000000000000000000000000000000000000000000000000000000000000000000000000000000000000000000000000000000001EFEE5
:3C37C800000000000000000000000000000000000000000000000000000000000000000000000000000000000000000000000000000000000000000000001EFEA9
:3C380400000000000000000000000000000000000000000000000000000000000000000000000000000000000000000000000000000000000000000000001EFE6C
:3C384000000000000000000000000000000000000000000000000000000000000000000000000000000000000000000000000000000000000000000000001EFE30
:3C387C00000000000000000000000000000000000000000000000000000000000000000000000000000000000000000000000000000000000000000000001EFEF4
:3C38B800000000000000000000000000000000000000000000000000000000000000000000000000000000000000000000000000000000000000000000001EFEB8
:3C38F400000000000000000000000000000000000000000000000000000000000000000000000000000000000000000000000000000000000000000000001EFE7C
:3C393000020000000000000000000000000000000000000000000000000000000000000000000000000000000000000000000000000000000000000000002FFF2B
:3C396C00020000000000000000000000000000000000000000000000000000000000000000000000000000000000000000000000000000000000000000002FFFEF
:3C39A800000000000000000000000000000000000000000000000000000000000000000000000000000000000000000000000000000000000000000000001EFEC7
:3C39E400020000000000000000000000000000000000000000000000000000000000000000000000000000000000000000000000000000000000000000002FFF77
:3C3A2000020000000000000000000000000000000000000000000000000000000000000000000000000000000000000000000000000000000000000000002FFF3A
:3C3A5C00000000000000000000000000000000000000000000000000000000000000000000000000000000000000000000000000000000000000000000001EFE12
:3C3A9800000000000000000000000000000000000000000000000000000000000000000000000000000000000000000000000000000000000000000000001EFED6
:3C3AD400000000000000000000000000000000000000000000000000000000000000000000000000000000000000000000000000000000000000000000001EFE9A
:3C3B1000020000000000000000000000000000000000000000000000000000000000000000000000000000000000000000000000000000000000000000002FFF49
:3C3B4C00020000000000000000000000000000000000000000000000000000000000000000000000000000000000000000000000000000000000000000002FFF0D
:3C3B8800020000000000000000000000000000000000000000000000000000000000000000000000000000000000000000000000000000000000000000003EFEC3
:3C3BC400000000000000000000000000000000000000000000000000000000000000000000000000000000000000000000000000000000000000000000000FFFB7
:3C3C0000000000000000000000000000000000000000000000000000000000000000000000000000000000000000000000000000000000000000000000000FFF7A
:3C3C3C00000000000000000000000000000000000000000000000000000000000000000000000000000000000000000000000000000000000000000000000FFF3E
:3C3C7800000000000000000000000000000000000000000000000000000000000000000000000000000000000000000000000000000000000000000000001EFEF4
:3C3CB400000000000000000000000000000000000000000000000000000000000000000000000000000000000000000000000000000000000000000000001EFEB8
:3C3CF000020000000000000000000000000000000000000000000000000000000000000000000000000000000000000000000000000000000000000000002FFF68
:3C3D2C00020000000000000000000000000000000000000000000000000000000000000000000000000000000000000000000000000000000000000000002FFF2B
:3C3D6800020000000000000000000000000000000000000000000000000000000000000000000000000000000000000000000000000000000000000000002FFFEF
:3C3DA400000000000000000000000000000000000000000000000000000000000000000000000000000000000000000000000000000000000000000000000FFFD5
:3C3DE000000000000000000000000000000000000000000000000000000000000000000000000000000000000000000000000000000000000000000000000FFF99
:3C3E1C00000000000000000000000000000000000000000000000000000000000000000000000000000000000000000000000000000000000000000000000FFF5C
:3C3E5800000000000000000000000000000000000000000000000000000000000000000000000000000000000000000000000000000000000000000000001EFE12
:3C3E9400000000000000000000000000000000000000000000000000000000000000000000000000000000000000000000000000000000000000000000001EFED6
:3C3ED000020000000000000000000000000000000000000000000000000000000000000000000000000000000000000000000000000000000000000000002FFF86
:3C3F0C00020000000000000000000000000000000000000000000000000000000000000000000000000000000000000000000000000000000000000000002FFF49
:3C3F4800020000000000000000000000000000000000000000000000000000000000000000000000000000000000000000000000000000000000000000002FFF0D
:3C3F8400000000000000000000000000000000000000000000000000000000000000000000000000000000000000000000000000000000000000000000000FFFF3
:3C3FC000000000000000000000000000000000000000000000000000000000000000000000000000000000000000000000000000000000000000000000000FFFB7
:3C3FFC00000000000000000000000000000000000000000000000000000000000000000000000000000000000000000000000000000000000000000000000FFF7B
:3C403800000000000000000000000000000000000000000000000000000000000000000000000000000000000000000000000000000000000000000000001EFE30
:3C407400000000000000000000000000000000000000000000000000000000000000000000000000000000000000000000000000000000000000000000001EFEF4
:3C40B000020000000000000000000000000000000000000000000000000000000000000000000000000000000000000000000000000000000000000000002FFFA4
:3C40EC00020000000000000000000000000000000000000000000000000000000000000000000000000000000000000000000000000000000000000000002FFF68
:3C412800020000000000000000000000000000000000000000000000000000000000000000000000000000000000000000000000000000000000000000002FFF2B
:3C416400000000000000000000000000000000000000000000000000000000000000000000000000000000000000000000000000000000000000000000000FFF11
:3C41A000000000000000000000000000000000000000000000000000000000000000000000000000000000000000000000000000000000000000000000000FFFD5
:3C41DC00000000000000000000000000000000000000000000000000000000000000000000000000000000000000000000000000000000000000000000000FFF99
:3C421800000000000000000000000000000000000000000000000000000000000000000000000000000000000000000000000000000000000000000000001EFE4E
:3C425400000000000000000000000000000000000000000000000000000000000000000000000000000000000000000000000000000000000000000000001EFE12
:3C429000020000000000000000000000000000000000000000000000000000000000000000000000000000000000000000000000000000000000000000002FFFC2
:3C42CC00020000000000000000000000000000000000000000000000000000000000000000000000000000000000000000000000000000000000000000002FFF86
:3C430800020000000000000000000000000000000000000000000000000000000000000000000000000000000000000000000000000000000000000000002FFF49
:3C434400000000000000000000000000000000000000000000000000000000000000000000000000000000000000000000000000000000000000000000000FFF2F
:3C438000000000000000000000000000000000000000000000000000000000000000000000000000000000000000000000000000000000000000000000000FFFF3
:3C43BC00000000000000000000000000000000000000000000000000000000000000000000000000000000000000000000000000000000000000000000001EFEA9
:3C43F800000000000000000000000000000000000000000000000000000000000000000000000000000000000000000000000000000000000000000000001EFE6D
:3C443400000000000000000000000000000000000000000000000000000000000000000000000000000000000000000000000000000000000000000000001EFE30
:3C447000020000000000000000000000000000000000000000000000000000000000000000000000000000000000000000000000000000000000000000002FFFE0
:3C44AC00020000000000000000000000000000000000000000000000000000000000000000000000000000000000000000000000000000000000000000002FFFA4
:3C44E800000000000000000000000000000000000000000000000000000000000000000000000000000000000000000000000000000000000000000000001EFE7C
:3C452400020000000000000000000000000000000000000000000000000000000000000000000000000000000000000000000000000000000000000000002FFF2B
:3C456000020000000000000000000000000000000000000000000000000000000000000000000000000000000000000000000000000000000000000000002FFFEF
:3C459C00000000000000000000000000000000000000000000000000000000000000000000000000000000000000000000000000000000000000000000000FFFD5
:3C45D800000000000000000000000000000000000000000000000000000000000000000000000000000000000000000000000000000000000000000000001EFE8B
:3C461400000000000000000000000000000000000000000000000000000000000000000000000000000000000000000000000000000000000000000000001EFE4E
:3C465000020000000000000000000000000000000000000000000000000000000000000000000000000000000000000000000000000000000000000000003EFEF0
:3C468C00020000000000000000000000000000000000000000000000000000000000000000000000000000000000000000000000000000000000000000002FFFC2
:3C46C800020000000000000000000000000000000000000000000000000000000000000000000000000000000000000000000000000000000000000000002FFF86
:3C470400000000000000000000000000000000000000000000000000000000000000000000000000000000000000000000000000000000000000000000001EFE5D
:3C474000000000000000000000000000000000000000000000000000000000000000000000000000000000000000000000000000000000000000000000001EFE21
:3C477C00000000000000000000000000000000000000000000000000000000000000000000000000000000000000000000000000000000000000000000000FFFF3
:3C47B800000000000000000000000000000000000000000000000000000000000000000000000000000000000000000000000000000000000000000000001EFEA9
:3C47F400000000000000000000000000000000000000000000000000000000000000000000000000000000000000000000000000000000000000000000001EFE6D
:3C483000020000000000000000000000000000000000000000000000000000000000000000000000000000000000000000000000000000000000000000003EFE0E
:3C486C00020000000000000000000000000000000000000000000000000000000000000000000000000000000000000000000000000000000000000000002FFFE0
:3C48A800020000000000000000000000000000000000000000000000000000000000000000000000000000000000000000000000000000000000000000002FFFA4
:3C48E400000000000000000000000000000000000000000000000000000000000000000000000000000000000000000000000000000000000000000000000FFF8A
:3C492000000000000000000000000000000000000000000000000000000000000000000000000000000000000000000000000000000000000000000000000FFF4D
:3C495C00020000000000000000000000000000000000000000000000000000000000000000000000000000000000000000000000000000000000000000002FFFEF
:3C499800000000000000000000000000000000000000000000000000000000000000000000000000000000000000000000000000000000000000000000001EFEC7
:3C49D400000000000000000000000000000000000000000000000000000000000000000000000000000000000000000000000000000000000000000000001EFE8B
:3C4A1000000000000000000000000000000000000000000000000000000000000000000000000000000000000000000000000000000000000000000000001EFE4E
:3C4A4C00000000000000000000000000000000000000000000000000000000000000000000000000000000000000000000000000000000000000000000001EFE12
:3C4A8800008000800080008000800080008000800080008000800080008000800080008000800080008000800080008000800080008000800080008000009EFE56
:3C4AC400000000000000000000000000000000000000000000000000000000000000000000000000000000000000000000000000000000000000000000001EFE9A
:3C4B0000000000000000000000000000000000000000000000000000000000000000000000000000000000000000000000000000000000000000000000001EFE5D
:3C4B3C00000000000000000000000000000000000000000000000000000000000000000000000000000000000000000000000000000000000000000000001EFE21
:3C4B7800000000000000000000000000000000000000000000000000000000000000000000000000000000000000000000000000000000000000000000001EFEE5
:3C4BB400000000000000000000000000000000000000000000000000000000000000000000000000000000000000000000000000000000000000000000001EFEA9
:3C4BF000000000000000000000000000000000000000000000000000000000000000000000000000000000000000000000000000000000000000000000001EFE6D
:3C4C2C00000000000000000000000000000000000000000000000000000000000000000000000000000000000000000000000000000000000000000000001EFE30
:3C4C6800000000000000000000000000000000000000000000000000000000000000000000000000000000000000000000000000000000000000000000001EFEF4
:3C4CA400000000000000000000000000000000000000000000000000000000000000000000000000000000000000000000000000000000000000000000001EFEB8
:3C4CE000000000000000000000000000000000000000000000000000000000000000000000000000000000000000000000000000000000000000000000001EFE7C
:3C4D1C00000000000000000000000000000000000000000000000000000000000000000000000000000000000000000000000000000000000000000000001EFE3F
:3C4D5800000000000000000000000000000000000000000000000000000000000000000000000000000000000000000000000000000000000000000000001EFE03
:3C4D9400000000000000000000000000000000000000000000000000000000000000000000000000000000000000000000000000000000000000000000001EFEC7
:3C4DD000000000000000000000000000000000000000000000000000000000000000000000000000000000000000000000000000000000000000000000001EFE8B
:3C4E0C00000000000000000000000000000000000000000000000000000000000000000000000000000000000000000000000000000000000000000000001EFE4E
:3C4E4800000000000000000000000000000000000000000000000000000000000000000000000000000000000000000000000000000000000000000000001EFE12
:3C4E8400000000000000000000000000000000000000000000000000000000000000000000000000000000000000000000000000000000000000000000001EFED6
:3C4EC000000000000000000000000000000000000000000000000000000000000000000000000000000000000000000000000000000000000000000000001EFE9A
:3C4EFC00000000000000000000000000000000000000000000000000000000000000000000000000000000000000000000000000000000000000000000001EFE5E
:3C4F3800000000000000000000000000000000000000000000000000000000000000000000000000000000000000000000000000000000000000000000001EFE21
:3C4F7400000000000000000000000000000000000000000000000000000000000000000000000000000000000000000000000000000000000000000000001EFEE5
:3C4FB000000000000000000000000000000000000000000000000000000000000000000000000000000000000000000000000000000000000000000000001EFEA9
:3C4FEC00000000000000000000000000000000000000000000000000000000000000000000000000000000000000000000000000000000000000000000001EFE6D
:3C502800000000000000000000000000000000000000000000000000000000000000000000000000000000000000000000000000000000000000000000001EFE30
:3C506400000000000000000000000000000000000000000000000000000000000000000000000000000000000000000000000000000000000000000000001EFEF4
:3C50A000000000000000000000000000000000000000000000000000000000000000000000000000000000000000000000000000000000000000000000001EFEB8
:3C50DC00000000000000000000000000000000000000000000000000000000000000000000000000000000000000000000000000000000000000000000001EFE7C
:3C511800000000000000000000000000000000000000000000000000000000000000000000000000000000000000000000000000000000000000000000001EFE3F
:3C515400000000000000000000000000000000000000000000000000000000000000000000000000000000000000000000000000000000000000000000001EFE03
:3C519000000000000000000000000000000000000000000000000000000000000000000000000000000000000000000000000000000000000000000000001EFEC7
:3C51CC00000000000000000000000000000000000000000000000000000000000000000000000000000000000000000000000000000000000000000000001EFE8B
:3C520800000000000000000000000000000000000000000000000000000000000000000000000000000000000000000000000000000000000000000000001EFE4E
:3C524400000000000000000000000000000000000000000000000000000000000000000000000000000000000000000000000000000000000000000000001EFE12
:3C528000000000000000000000000000000000000000000000000000000000000000000000000000000000000000000000000000000000000000000000001EFED6
:3C52BC00000000000000000000000000000000000000000000000000000000000000000000000000000000000000000000000000000000000000000000001EFE9A
:3C52F800000000000000000000000000000000000000000000000000000000000000000000000000000000000000000000000000000000000000000000001EFE5E
:3C533400000000000000000000000000000000000000000000000000000000000000000000000000000000000000000000000000000000000000000000001EFE21
:3C537000000000000000000000000000000000000000000000000000000000000000000000000000000000000000000000000000000000000000000000001EFEE5
:3C53AC00000000000000000000000000000000000000000000000000000000000000000000000000000000000000000000000000000000000000000000000FFFB7
:3C53E800000000000000000000000000000000000000000000000000000000000000000000000000000000000000000000000000000000000000000000001EFE6D
:3C542400000000000000000000000000000000000000000000000000000000000000000000000000000000000000000000000000000000000000000000001EFE30
:3C546000020000000000000000000000000000000000000000000000000000000000000000000000000000000000000000000000000000000000000000003EFED2
:3C549C00020000000000000000000000000000000000000000000000000000000000000000000000000000000000000000000000000000000000000000002FFFA4
:3C54D800000000000000000000000000000000000000000000000000000000000000000000000000000000000000000000000000000000000000000000000FFF8A
:3C551400020000000000000000000000000000000000000000000000000000000000000000000000000000000000000000000000000000000000000000002FFF2B
:3C555000020000000000000000000000000000000000000000000000000000000000000000000000000000000000000000000000000000000000000000002FFFEF
:3C558C0002000000000000000000000000000000000000000000000000000000000000000000000000000000000000000000000000000000000000800E0041FF13
:3C55C8000000000000000000000000000000000000000000000000000000000000000000000000000000000000000000000000000000000000000000060078FE2B
:3C560400000000000000000000000000000000000000000000000000000000000000000000000000000000000000000000000000000000000000000000001EFE4E
:3C56400002000000000000000000000000000000000000000000000000000000000000000000000000000000000000000000000000000000000000802000BCFED2
:3C567C00020000000000000000000000000000000000000000000000000000000000000000000000000000000000000000000000000000000000000000002FFFC2
:3C56B800020000000000000000000000000000000000000000000000000000000000000000000000000000000000000000000000000000000000000000002FFF86
:3C56F40002000000000000000000000000000000000000000000000000000000000000000000000000000000000000000000000000000000000000800600D8FE1C
:3C5730000200000000000000000000000000000000000000000000000000000000000000000000000000000000000000000000000000000000000000060058FEDF
:3C576C0000000000000000000000000000000000000000000000000000000000000000000000000000000000000000000000000000800C00000000880600BCFE2D
:3C57A800000000000000000000000000000000000000000000000000000000000000000000000000000000000000000000000000000004000000000006003CFE81
:3C57E40000000000000000000000000000000000000000000000000000000000000000000000000000000000000000000000000000800200000000000600DAFE29
:3C58200002000000000000000000000000000000000000000000000000000000000000000000000000000000000000000000000000802200000000C036003BFE79
:3C585C0002000000000000000000000000000000000000000000000000000000000000000000000000000000000000000000000000800C0000000030060035FF18
:3C589800000000000000000000000000000000000000000000000000000000000000000000000000000000000000000000000000000002000000000006005AFE74
:3C58D40002000000000000000000000000000000000000000000000000000000000000000000000000000000000000000000000000000200000000800600EBFF24
:3C591000020000000000000000000000000000000000000000000000000000000000000000000000000000000000000000000000000024000000000012105BFFB9
:3C594C000200000000000000000000000000000000000000000000000000000000000000000000000000000000000000000000000080120000000080040059FEB0
:3C5988000000000000000000000000000000000000000000000000000000000000000000000000000000000000000000000000000000020000000000040078FE67
:3C59C400000000000000000000000000000000000000000000000000000000000000000000000000000000000000000000000000008002000000008002001EFE87
:3C5A0000020000000000000000000000000000000000000000000000000000000000000000000000000000000000000000000000008022000000008002003CFE0A
:3C5A3C000200000000000000000000000000000000000000000000000000000000000000000000000000000000000000000000000080120000000080140049FFBE
:3C5A78000200000000000000000000000000000000000000000000000000000000000000000000000000000000000000000000000000040000000000020049FFA2
:3C5AB400020000000000000000000000000000000000000000000000000000000000000000000000000000000100000000000000000002000000000002002EFF82
:3C5AF00002000000000000000000000000000000000000000000000000000000000000000000000000000080000000000000000000002400000000002400B6FEFC
:3C5B2C0002000000000000000000000000000000000000000000000000000000000000A406000000000000000000000000000000000000000000008000007CFE97
:3C5B68000000000000000000000000000000000000000000000000000000000000000000060000000000000000000000000000000000000000000000000078FE85
:3C5BA40000000000000000000000000000000000000000000000000000000000000000000600000000000000000000000000000000000000000000800200DAFE65
:3C5BE000020000000000000000000000000000000000000000000000000000000000008056000000000000000000000000000000000000000000008002007FFEB2
:3C5C1C0002000000000000000000000000000000000000000000000000000000000000410000000000000000000000000000000000000000000000800400BBFECC
:3C5C5800020000000000000000000000000000000000000000000000000000000000000006000000000000000000000000000000000000000000000002007AFE8E
:3C5C940002000000000000000000000000000000000000000000000000000000000000800600000000000000000001000000000000000000000000000200FBFF4F
:3C5CD0001201000000000000000000000000000000000000000000000000000000000000060000000000000000800000000000000000000000000000340007FEC6
:3C5D0C0002000000000000000000000000000000000000000000000000000000000000000000000000000000000000000000000000000000009000800000B7FE94
:3C5D4800008000000000000000000000000000000000000000000000000000000000000000000000000000000000000000000000000000000000000000009EFE03
:3C5D840000000000000000000000000000000000000000000000000000000000000000000000000000000000000000000000000000000000008006800200D4FE09
:3C5DC0000200000000000000000000000000000000000000000000000000000000000000000000000000000000000000000000000000000000A006800200F6FE89
:3C5DFC0002000000000000000000000000000000000000000000000000000000000000000000000000000000000000000000000000000000008000800400E3FF83
:3C5E3800020000000000000000000000000000000000000000000000000000000000000000000000000000000000000000000000000000000000000002000DFF1E
:3C5E7400020000000000000000000000000000000000000000000000000000000000000000000000000000000000000000000000000000000000060002007CFE6E
:3C5EB000028000000000000000000000000000000000000000000000000000000000000000000000000000000000000000000000000000000000060014108AFE82
:3C5EEC000800000000000000000000000000000000000000000000000000000000000000000000000000000000000000000000000000000000800080000007FF6C
:3C5F2800000000000000000000000000000000000000000000000000000000000000000000000000000000000000000000000000000000000000000000001EFE21
:3C5F64000000000000000000000000000000000000000000000000000000000000000000000000000000000000000000000000000000000000800680060090FE67
:3C5FA00002040000000000000000000000000000000000000000000000000000000000000000000000000000000000000000000000000000008000800000B2FE0F
:3C5FDC000200000000000000000000000000000000000000000000000000000000000000000000000000000000000000000000000000000000B000B0000085FEA4
:3C6018000200000000000000000000000000000000000000000000000000000000000000000000000000000000000000000000000000000000000600060029FF16
:3C6054000200000000000000000000000000000000000000000000000000000000000000000000000000000000000000000000000000000000000600060038FECC
:3C609000500000000000000000000000000000000000000000000000000000000000000000000000000000000000000000000000000000000000000000005AFF2B
:3C60CC000000000000000000000000000000000000000000000000000000000000000000000000000000000000000000000000000000000000800080000096FE04
:3C610800000000000000000000000000000000000000000000000000000000000000000000000000000000000000000000000000000000000000000000001EFE3F
:3C6144000000000000000000000000000000000000000000000000000000000000000000000000000000000000000000000000000000000000800680060090FE85
:3C61800002000000000000000000000000000000000000000000000000000000000000000000000000000000000000000000000000000000008000800000A7FF3B
:3C61BC000200000000000000000000000000000000000000000000000000000000000000000000000000000000000000000000000000000000D000D00000E3FE24
:3C61F8000000000000000000000000000000000000000000000000000000000000000000000000000000000000000000000000000000000000000600060018FE49
:3C6234000200000000000000000000000000000000000000000000000000000000000000000000000000000000000000000000000000000000000600060029FFF8
:3C627000020000000000000000000000000000000000000000000000000000000000000000000000000000000000000000000000000000000000000000002FFFC2
:3C62AC0000000000000000000000000000000000000000000000000000000000000000A20600000000000000000000000000000000840000008000800000C7FFC4
:3C62E800000000000000000000000000000000000000000000000000000000000000000006000000000000000000000000000000000006000000000000001EFE52
:3C63240000000000000000000000000000000000000000000000000000000000000000000600000000000000000000000000000000000000008006800600F6FE37
:3C63600002000000000000000000000000000000000000000000000000000000000000800E02000000000000000000000000000000A0060000800680060038FE87
:3C639C0002000000000000000000000000000000000000000000000000000000000000080C0000000000000000000000000000000042000000800680060027FF3B
:3C63D8000200000000000000000000000000000000000000000000000000000000000000060000000000000000000000000000000000060000000600060029FF47
:3C6414000000000000000000000000000000000000000000000000000000000000000080060000000100000000000100010000000080000000000000000078FFCC
:3C64500000000000000000000000000000000000000000000000000000000000000000408600008000000000008000800000000000000600000000000000D6FEF0
:3C648C0000000000000000000000000000000000000000000000000000000000000080801600000000000000000000000000000000000000000000D01600D7FF02
:3C64C800000000000000000000000000000000000000000000000000000000000000000006000000000000000000000000000000000000000000000006001EFE70
:3C6504000000000000000000000000000000000000000000000000000000000000000000060000000000000000000000000000000000000000000000000078FEDF
:3C65400002000000000000000000000000000000000000000000000000000000000000A0860000000000000000000000000000000000000000000080260014FE3F
:3C657C00020000000000000000000000000000000000000000000000000000000000000804000000000000000000000000000000000800000000001006001DFF9B
:3C65B8000080008000800080008000800080008000800080008000800080008000800080068000800080008000800080008000800080008000000000060007FF95
:3C65F400020000000000000000000000000000000000000000000000000000000000000006000000010001000000000000000100000000000000000006003EFE1E
:3C66300002000000000000000000000000000000000000000000000000000000000000203600008000800000000000000080000000200000000000C02F0066FEE3
:3C666C0000000000000000000000000000000000000000000000000000000000000000000000000000000000000000000000000000420100000000800001CCFF63
:3C66A800000000000000000000000000000000000000000000000000000000000000000000000000000000000000000000000000000800000020000800001CFE6C
:3C66E400000000000000000000000000000000000000000000000000000000000000000000000000000000000000000000000000000000000000000000001EFE5E
:3C672000000000000000000000000000000000000000000000000000000000000000000000000000000000000000000000000000000000000000000000001EFE21
:3C675C00000000000000000000000000000000000000000000000000000000000000000000000000000000000000000000000000000000000000000000001EFEE5
:3C679800000000000000000000000000000000000000000000000000000000000000000020000000000000000000000000000000000000000000000000000DFF99
:3C67D400000000000000000000000000000000000000000000000000000000000000002000000000000000000000000002000000000000000000000000001CFE4D
:3C6810000000000000000000000000000000000000000000000000000000000000000000080800000400000000000100000000000000000000000000000046FEF3
:3C684C00000000000000000000000000000000000000000000000000000000000000002000000000000000000100000000000000000000000000000000002EFFC2
:3C688800000000000000000000000000000000000000000000000000000000000000000300000000020000000000040000000000000000000000000000006CFF60
:3C68C400000000000000000000000000000000000000000000000000000000000000000000000000000000000000000000000000000000000000000000001EFE7C
:3C690000000000000000000000000000000000000000000000000000000000000000000000000000000000000000000000000000000000000000000000001EFE3F
:3C693C00000000000000000000000000000000000000000000000000000000000000000000000000000000000000000000000000000000000000000000001EFE03
:3C69780000100000000000000000000000000000000000000000000000000000000000000800000000000000000000000000040000000000000000000400C6FEFF
:3C69B40000000000000000000000000000000000000000000000000000000000000008000000000000000400000000000000000000000000000000000000DAFEC3
:3C69F000000000000000000000000000000000000000000000000000000000000000000000000000000000000000000000000000004000000000010000004EFEDE
:3C6A2C00000000000000000000000000000000000000000000000000000000000000000000000000000000000000000000000000000000000000000000001EFE12
:3C6A6800000000000000000000000000000000000000000000000000000000000000000000000000000000000000000000000000000000000000000000001EFED6
:3C6AA40000000000000000000000000000000000000000000000000000000000000000000000000000000000000000000000000000200000000000000800B6FEDA
:3C6AE000000000000000000000000000000000000000000000000000000000000000000000000000000000000000000000000000000000000000000000001EFE5E
:3C6B1C00000000000000000000000000000000000000000000000000000000000000000000000000000000000000000000000000000000000000000000001EFE21
:3C6B5800000000000000000000000000000000000000000000000000000000000000000000000000000000000000000000000000000000000000000000001EFEE5
:3C6B9400000000000000000000000000000000000000000000000000000000000000000000000000000000000000000000000000000000000000000000001EFEA9
:3C6BD000000000000000000000000000000000000000000000000000000000000000000000000000000000000000000000000000000000000000000000001EFE6D
:3C6C0C00000000000000000000000000000000000000000000000000000000000000000000000000000000000000000000000000000000000000000000001EFE30
:3C6C4800000000000000000000000000000000000000000000000000000000000000000000000000000000000000000000000000000000000000000000001EFEF4
:3C6C8400000000000000000000000000000000000000000000000000000000000000000000000000000000000000000000000000000000000000000000001EFEB8
:3C6CC000000000000000000000000000000000000000000000000000000000000000000000000000000000000000000000000000000000000000000000001EFE7C
:3C6CFC00000100000000000000000000000000000000000000000000000000000000000000000000000000000000000000000000001000000000000000001EFF2E
:3C6D3800000000000000000000000000000000000000000000000000000000000000000000000000000000000000000000000000000000000000000000001EFE03
:3C6D7400080000010000000000000000000000000000000000000000000000000000000000000000000000000000000000000000000000000000000000008EFE4E
:3C6DB000000000000000000000000000000000000000000000000000000000000000000000000000000000000000000000000000000000000000000000001EFE8B
:3C6DEC00000000000000000000000000000000000000000000000000000000000000000000000000000000000000000000000000000000000000000000001EFE4F
:3C6E28000000000000000000000000000000000000000000000000000000000000000000000000000000000000000000000000000002080000000000000094FE92
:3C6E6400000000000000000000000000000000000000000000000000000000000000000800000000000000000000000000000000000804000000000000005AFE86
:3C6EA000000000000000000000000000000000000000000000000000000000000000000000000000000000000000000000000000000000000000000000001EFE9A
:3C6EDC000200000000000000000000000000000000000000000000000000000000D0120000800000000000000000000000000000000000000000000000009BFF7C
:3C6F1800000000000000000000000000000000000000000000000000000000000000060000000000000000000000000000000000000000000000000000007EFEBB
:3C6F540000000000000000000000000000000000000000000000000000000000000006000080020000000000000000000000000000000000000000000000F4FE87
:3C6F900000000000000000000000000000000000000000000000000000000000008006010080020000000000000000000000000000000000000000000000ECFFD1
:3C6FCC000000000000000000000000000000000000000000000000000000000000100E00008004000000000000000000000000000000000000000000000062FF86
:3C700800000000000000000000000000000000000000000000000000000000000000060000000200000000000000000000000000000000000000000000007CFECA
:3C7044000000000000000000000000000000000000000000000000000000000000800600000002000000000000000000000000000000000000000000000074FE16
:3C708000008001000000000000000000000000000000000000000000000000000040060100004C0000000000000000000000000000000000000000000000A6FE1C
:3C70BC000800000000000000000000000000000000000000000000000000000000A1160000800000000000000000000000000000000000000000000000007CFEDF
:3C70F800000000000000000000000000000000000000000000000000000000000000060000000000000000000000000000000000000000000000000000007EFEDA
:3C71340000000000000000000000000000000000000000000000000000000000000006000080020000000000000000000000000000000000000000000000F4FEA5
:3C71700002040000000000000000000000000000000000000000000000000000008026000080020000000000000000000000000000000000000000000000EBFFCB
:3C71AC0002000000000000000000000000000000000000000000000000000000000216000080040000000000000000000000000000000000000000000000E1FE2A
:3C71E800020000000000000000000000000000000000000000000000000000000000020000000200000000000000000000000000000000000000000000001CFE4B
:3C7224000200010000000000000000000000000000000000000000000000000000800600000002000000000000000000000000000100010000000000000055FF4D
:3C726000888000000000000000000000000000000000000000000000000000000040060200002C000000000000000000000000800080000000000000000045FF32
:3C729C000800000000000000000000000000000000000000000000000000000000A40600008000000000000000000000000000000000000000000000000038FE4E
:3C72D800000000000000000000000000000000000000000000000000000000000000060000000000000000000000000000000000000000000000000000007EFEF8
:3C73140000000000000000000000000000000000000000000000000000000000000006000080020000000000000000000000000000000000000000000000F4FEC3
:3C7350000204000000000000000000000000000000000000000000000000000000802E0000800200000000000000000000000000000000000000000000006BFF61
:3C738C000A0000000000000000000000000000000000000000000000000000000008040000800C0000000000000000000000000000000000000000000000E3FF41
:3C73C800020000000000000000000000000000000000000000000000000000000000060000000200000000000000000000000000000000000000000000005CFE25
:3C7404000200000000000000000000000000000000000000000000000000000000800600000002000000000000000000000000000000000000000000000045FF7E
:3C7440008000000000000000000000000000000000000000000000000000000000404E00000024000000000000000000000000000000000000000000000003FFDC
:3C747C0000000000000000000000000000000000000000000000000000000000008004000080000000000000000000000000000000000000000000000000DEFEF4
:3C74B800000000000000000000000000000000000000000000000000000000000000040000000000000000000000000000000000000000000000000000005EFE38
:3C74F40000000000000000000000000000000000000000000000000000000000008002000080020000000000000000000000000000000000000000000000BCFE9E
:3C753000020000000000000000000000000000000000000000000000000000000080020000800200000000000000000000000000000000000000000000008DFF8D
:3C756C0002000000000000000000000000000000000000000000000000000000008014000080140000000000000000000000000000000000000000000000FBFEC0
:3C75A800000000000000000000000000000000000000000000000000000000000000020000000200000000000000000000000000000000000000000000003CFE69
:3C75E400020000000000000000000000000000000000000000000000000000000000020000000200000000000000000000000000000000000000000000000DFF59
:3C76200002800100000000000000000000000000000000000000000000000000000024000000240000000000000000000000000000000000000000000000E9FE7C
:3C765C00080000000000000000000000000000000000000000000000000000000080000000800000000000000000000000000000000000000000000000001EFECE
:3C769800000000000000000000000000000000000000000000000000000000000000000000000000000000000000000000000000000000000000000000001EFE9A
:3C76D40000000000000000000000000000000000000000000000000000000000008002000080020000000000000000000000000000000000000000000000BCFEBC
:3C7710000204000000000000000000000000000000000000000000000000000000800200008002000000000000000000000000000000000000000000000089FFAB
:3C774C000A0000000000000000000000000000000000000000000000000000000080040000800400000000000000000000000000000000000000000000006BFF85
:3C778800020000000000000000000000000000000000000000000000000000000000020000000200000000000000000000000000000000000000000000001CFEA5
:3C77C400020001000000000000000000000000000000000000000000000000000000020000000200000000000000000000000000010000000000000000001DFE66
:3C78000000820000000000000000000000000000000000000000000000000000000034000000340000000000000000000000008000000000000000000000D3FE11
:3C783C00080000000000000000000000000000000000000000000000000000000080000000800000000000000000000000000000000000000000000000001EFEEC
:3C787800000000000000000000000000000000000000000000000000000000000000000000000000000000000000000000000000000000000000000000001EFEB8
:3C78B40000000000000000000000000000000000000000000000000000000000008006000080060000000000000000000000000000000000000000000000F8FE96
:3C78F00002040000000000000000000000000000000000000000000000000000008000000080000000000000000000000000000000000000000000000000ABFFAC
:3C792C0002000000000000000000000000000000000000000000000000000000009000000090000000000000000000000000000000000000000000000000BFFF3F
:3C7968000200000000000000000000000000000000000000000000000000000000000600000006000000000000000000000000000000000000000000000058FE7F
:3C79A4000200000000000000000000000000000000000000000000000000000000000600000006000000000000000000000000000000000000000000000049FF51
:3C79E000100400000000000000000000000000000000000000000000000000000020000000200000000000000000000000000000000000000000000000002BFEEE
:3C7A1C00000000000000000000000000000000000000000000000000000000000080000000800000000000000000000000000000000000000000000000282DFFDA
:3C7A5800000000000000000000000000000000000000000000000000000000000000000000000000000000000000000000000000000000000000000000001EFED6
:3C7A940000000000000000000000000000000000000000000000000000000000008006000080060000000000000000000000000000000000000000000000F8FEB4
:3C7AD00002000000000000000000000000000000000000000000000000000000008000000080000000000000000000000000000000000000000000000000AFFFCA
:3C7B0C000200000000000000000000000000000000000000000000000000000000B0000000B00000000000000000000000000000000000000000000000081FFFB5
:3C7B48000000000000000000000000000000000000000000000000000000000000000600000006000000000000000000000000000000000000000000000069FF8D
:3C7B84000200000000000000000000000000000000000000000000000000000000000600000006000000000000000000000000000000000000000000000049FF6F
:3C7BC00002000000000000000000000000000000000000000000000000000080010000000080010000000000000000000000000000800100000000000040FAFFCB
:3C7BFC0000000000000000000000000000000000000000000000000000000000008000000080000000000088060000000000000000000000000080A00E0056FE3D
:3C7C3800000000000000000000000000000000000000000000000000000000000000000000000000000000000600000000000000000000000000000006007EFE88
:3C7C7400000000000000000000000000000000000000000000000000000000000080060000800600000000000600000000000000000000000000008002005CFEE6
:3C7CB000020000000000000000000000000000000000000000000000000000000080000000800000000000A0060000000000000000000000000000800210A1FEBF
:3C7CEC000200000000000000000000000000000000000000000000000000000000D0000000D00000000000000000000000000000000000000000008010006FFEBD
:3C7D28000000000000000000000000000000000000000000000000000000000000000600000006000000000000000000000000000000000000000000000078FE9D
:3C7D64000200010000000000000000000000000000000000000000000000000000000600000006000000008000000000000000000000000000000080020063FE71
:3C7DA00002800000000000000000000000000000000000000000000000000000000000000000000000000000000000000000000000000000000000000402CBFF55
:3C7DDC000800000000000000000000000000000000000000000000000000000000800000008000000000000000000000008416000000000000000090062885FF87
:3C7E180000800000000000000000000000000000000000000000000000000000000000000000000000000000000000000000060000000000000000000600FEFEA6
:3C7E5400000000000000000000000000000000000000000000000000000000000080060000800600000000000000000000000600000000000000008004003AFE24
:3C7E9000020400000000000000000000000000000000000000000000000000000080000000800600000000000000000000A0060400000000000000C05400D5FE19
:3C7ECC000200000000000000000000000000000000000000000000000000000000900000008006000000000000000000004114000000000000000080101069FE06
:3C7F0800020000000000000000000000000000000000000000000000000000000000060000000600000000000000000000000600000000000000000000004FFFDB
:3C7F44000200000000000000000000000000000000000000000000000000000000000600000000000000000000000000008006000000000000000080040005FFEB
:3C7F800090800000000000000000000000000000000000000000000000000000004000000000000000000000000000000000860000000000000000000242D2FFDA
:3C7FBC0008000000000000000000000000000000000000000000000000000000009006000000000000000000000000000000000000000000000000810028C5FF7E
:3C7FF8000000000000000000000000000000000000000000000000000000000000000600000000000000000000000000000000000000000000000000060018FE2B
:3C803400000000000000000000000000000000000000000000000000000000000000060000000000000000000000000000000000000000000000000000007EFE8E
:3C8070000204000000000000000000000000000000000000000000000000000000A036000000000000000000000000000000000000000000000000A00600A5FEAF
:3C80AC0002000000000000000000000000000000000000000000000000000000003008000000080000000000000000000000000000000000000000040050F5FF0E
:3C80E8000280008000800080008000800080008000800080008000800080008000800680000000800080008000800080008000800080008000800080060021FFAE
:3C812400020000000000000000000000000000000000000000000000000000000000060000000000000000000000000000000000000000000000000000004FFFC9
:3C81600010020000000000000000000000000000000000000000000000000000000006040000000400000000000000000000000000000000000000C007009AFE64
:3C819C00000000000000000000000000000000000000000000000000000000000080000100800001000000000000000000000000000000000000000000008EFE19
:3C81D800000000000000000000000000000000000000000000000000000000000020000000200000000000000000000000000000000000000000002000001EFEEF
:3C821400000000000000000000000000000000000000000000000000000000000000000000000000000000000000000000000000000000000000000000001EFE12
:3C825000000000000000000000000000000000000000000000000000000000000000000000000000000000000000000000000000000000000000000000001EFED6
:3C828C00000000000000000000000000000000000000000000000000000000000000000000000200000000000000000000200000000000000000000000003EFE58
:3C82C800000000000000000000000000000000000000000000000000000000000000000000000000000000000000000000000000000000000000000000001EFE5E
:3C830400000000000000000000000000000000000000000000000000000000000000000000000000000000000000000000000000000000000000000000001EFE21
:3C8340000000000000000000000000000000000000000000000000000000000000080000000004000000000000000000000000000100000000000800000002FEEC
:3C837C00000000000000000000000000000000000000000000000000000000000000000000000000000000000000000000000000000000000000000000001EFEA9
:3C83B8000000000000000000000000000000000000000000000000000000000000200000000000000000000000000000000004000000000000000000000018FE4F
:3C83F400000201000000000000000000000000000000000000000000000000000000000400000400000000000000000000000000000000000000000000001CFF27
:3C843000008400000000000000000000000000000000000000000000000000000000000000000000000000000000000000000000000000000000000000009AFEF4
:3C846C000000000000000000000000000000000000000000000000000000000000000000008000000000000000000000000100000000000000000000000086FECF
:3C84A800001000000000000000000000000000000000000000000000000000000000000000000000000000000000000000000000000000000000000004004AFE3C
:3C84E400000000000000000000000000000000000000000000000000000000000000000000000000000000000000000000000000000000000000000000001EFE40
:3C852000200002000000000000000000000000000000000000000000000000000000000100000100000000000000000000000000000000000000000000001EFEDF
:3C855C0000000000000000000000000000000000000000000000000000000000000080000000400000000000000000000000000000000000000000000000D6FE4F
:3C859800000000000000000000000000000000000000000000000000000000000000000000000000000000000000000000000000000000000000000000001EFE8B
:3C85D400000000000000000000000000000000000000000000000000000000000000100000000000000000200000000000000000000000000000000000003CFF00
:3C861000000000000000000000000000000000000000000000000000000000000000000000000000000000000000000000000000000000000000000000001EFE12
:3C864C00000000000000000000000000000000000000000000000000000000000000000000000000000000000000000000000000000000000000000000001EFED6
:3C868800000000000000000000000000000000000000000000000000000000000000000000000000000000000000000000000000000000000000000000001EFE9A
:3C86C40020080000000000000000000000000000000000000000000000000000000000000000000000000000000000000000000000100000000080000000ACFE18
:3C870000000000000000000000000000000000000000000000000000000000000000000000000000000000000000000000000000000000000000000000001EFE21
:3C873C000000000000000000000000000000000000000000000000000000000000000000004000000000000000000000000008000000000000000000000052FE69
:3C877800000000000000000000000000000000000000000000000000000000000000000000000000000000000000000000000000000000000000000000001EFEA9
:3C87B40000000000000000000000000000000000000000000000000000000000000000000004000000000000000000000000002800000000000000001000C4FF8A
:3C87F000000000000000000000000000000000000000000000000000000000000000001000002010000000400000000000000000000000000000000000043AFF90
:3C882C00000000000000000000000000000000000000000000000000000000000000000000000000000000000000000000000000000000000000000000001EFEF4
:3C88680000000000000000000000000000000000000000000000000000000000A00000000040000000000000000000000000000000000000000000000000EBFF0A
:3C88A400100200000000000000000000000000000000000000000000000000000000000000000000000000000000000000000000000000000000000000001CFF6B
:3C88E000000000000000000000000000000000000000000000000000000000000000000000000000000000000000000000000000000000000000000000001EFE40
:3C891C00000000000000000000000000000000000000000000000000000000000000000000000000000000000000000000000000000020000000001000000CFEE5
:3C895800002010000000000000000000000000000000000000000000000000000000000000000000000000000000000000000000000000000000000000002EFF86
:3C899400000000000000000000000000000000000000000000000000000000000000000000000000000000000000000000000000000000000000000000001EFE8B
:3C89D000000000000000000000000000000000000000000000000000000000000000080000000000000000000000000000000000000000000000000000009EFEC7
:3C8A0C0010000000000000000000000000000000000000000000000000000000000000000000000000000000000000000000000000000000000000000028ADFE4B
:3C8A4800000000000000000000000000000000000000000000000000000000000000000000000000000000000000000000000000000000000000000000001EFED6
:3C8A8400000000000000000000000000000000000000000000000000000000000000000000000000000000000000000000000000000000000000000000001EFE9A
:3C8AC0000208000000000000000000000000000000000000000000000000000000000000000000000000000000000000000000000000000000000000000027FF4A
:3C8AFC00020000000000000000000000000000000000000000000000000000000000000000000000000000000000000000000000000000000000000000506BFE83
:3C8B3800020000000000000000000000000000000000000000000000000000000000000000000000000000000000000000000000000000000000000000002FFFD1
:3C8B7400020000000000000000000000000000000000000000000000000000000000000000000000000000000000000000000000000000000000000000002FFF95
:3C8BB0000810000000000000000000000000000000000000000000000000000000000000000000000000000000000000000000800100000000000000000096FE5C
:3C8BEC0000800400000000000000000000000000000000000000000000000000000000000000000000000000000000000000000000000000000000000000DAFEF1
:3C8C2800000004000000000000000000000000000000000000000000000000000000000000000000000000000000000000000000000000000000000000005AFEB4
:3C8C640000800200000000000000000000000000000000000000000000000000000000000000000000000000000000000000000000000000000000000000BCFE98
:3C8CA000028002000000000000000000000000000000000000000000000000000000000000000000000000000000000000000000000000000000000000008DFF88
:3C8CDC0002800400000000000000000000000000000000000000000000000000000000000000000000000000000000000000000000000000000000000000EBFFEC
:3C8D1800000002000000000000000000000000000000000000000000000000000000000000000000000000000000000000000000000000000000000000003CFEE3
:3C8D5400020002000000000000000000000000000000000000000000000000000000000000000000000000000000000000000000000000000000000000000DFFD3
:3C8D900002002C00000000000000000000000000000000000000000000000000000000000000000000000000000000000000000000000000000000000000E1FF99
:3C8DCC00008000000000000000000000000000000000000000000000000000000000000000000000000000000000000000000000000000000000000000282DFF97
:3C8E0800000000000000000000000000000000000000000000000000000000000000000000000000000000000000000000000000000000000000000000001EFE12
:3C8E440000800200000000000000000000000000000000000000000000000000000000000000000000000000000000000000000000000000000000000000BCFEB6
:3C8E8000028002000000000000000000000000000000000000000000000000000000000000000000000000000000000000000000000000000000000000008DFFA6
:3C8EBC0002800C0000000000000000000000000000000000000000000000000000000000000000000000000000000000000000000000000000000000001063FE7B
:3C8EF800000002000000000000000000000000000000000000000000000000000000000000000000000000000000000000000000000000000000000000002DFF10
:3C8F3400020002000000000000000000000000000000000000000000000000000000000000000000000000000000000000000000000000000000000000000DFFF1
:3C8F7000020024000000000000000000000000000000000000000000000000000000000000000000000000000000000000000000000000000000000000205AFE27
:3C8FAC00028000000000000000000000000000000000000000000000000000000000000000000000000000000000000000000000000000000000000000280DFFD3
:3C8FE800000000000000000000000000000000000000000000000000000000000000000000000000000000000000000000000000000000000000000000001EFE31
:3C90240000800200000000000000000000000000000000000000000000000000000000000000000000000000000000000000000000000000000000000000BCFED4
:3C906000028002000000000000000000000000000000000000000000000000000000000000000000000000000000000000000000000000000000000000008DFFC4
:3C909C0012801400000000000000000000000000000000000000000000000000000000000000000000000000000000000000000000000000000000000030D9FEEB
:3C90D800020002000000000000000000000000000000000000000000000000000000000000000000000000000000000000000000000000000000000000000DFF4C
:3C911400020002000000000000000000000000000000000000000000000000000000000000000000000000000000000000000000000000000000000000000DFF0F
:3C9150000208240000000000000000000000000000000000000000000000000000000000000000000000000000000000000000800100000000000000000068FECE
:3C918C00008000000000000000000000000000000000000000000000000000000000000000000000000000000000000000000000000000000000000000009EFE8B
:3C91C800000000000000000000000000000000000000000000000000000000000000000000000000000000000000000000000000000000000000000000001EFE4F
:3C92040000800200000000000000000000000000000000000000000000000000000000000000000000000000000000000000000000000000000000000000BCFEF2
:3C924000028002000000000000000000000000000000000000000000000000000000000000000000000000000000000000000000000000000000000000008DFFE2
:3C927C0002800400000000000000000000000000000000000000000000000000000000000000000000000000000000000000000000000000000000000000EBFF46
:3C92B800000002000000000000000000000000000000000000000000000000000000000000000000000000000000000000000000000000000000000000003CFE3E
:3C92F400020002000000000000000000000000000000000000000000000000000000000000000000000000000000000000000000000000000000000000000DFF2E
:3C9330000200340000000000000000000000000000000000000000000000000000000000000000000000000000000000000000000000000000000000000079FE54
:3C936C0002800000000000000000000000000000000000000000000000000000000000000000000000000000000000000000000000000000000000A406007CFE1F
:3C93A8000000000000000000000000000000000000000000000000000000000000000000000000000000000000000000000000000000000000000000060078FE0D
:3C93E400008006000000000000000000000000000000000000000000000000000000000000000000000000000000000000000000000000000000008002005AFEED
:3C942000028000000000000000000000000000000000000000000000000000000000000000000000000000000000000000000000000000000000008012101DFFD0
:3C945C00029000000000000000000000000000000000000000000000000000000000000000000000000000000000000000000000000000000000008000003FFF84
:3C9498000200060000000000000000000000000000000000000000000000000000000000000000000000000000000000000000000000000000000000000058FE3A
:3C94D40002000600000000000000000000000000000000000000000000000000000000000000000000000000000000000000000000000000000000800200EBFFE8
:3C95100002200000000000000000000000000000000000000000000000000000000000000000000000000000000000000000000000000000000000000C0483FF6B
:3C954C0000800000000000000000000000000000000000000000000000000000000000000000000000000000000000000000000000000000000000B002000CFEA7
:3C958800000000000000000000000000000000000000000000000000000000000000000000000000000000000000000000000000000000000000000002003CFE6B
:3C95C400008006000000000000000000000000000000000000000000000000000000000000000000000000000000000000000000000000000000008006001EFE43
:3C96000002800000000000000000000000000000000000000000000000000000000000000000000000000000000000000000000000000000000000800E0481FF9A
:3C963C0002B000000000000000000000000000000000000000000000000000000000000000000000000000000000000000000000000000000000008010000FFEA3
:3C9678000000060000000000000000000000000000000000000000000000000000000000000000000000000000000000000000000000000000000000000078FE3A
:3C96B400020006000000000000000000000000000000000000000000000000000000000000000000000000000000000000000000000000000000008004008DFF62
:3C96F000020000000000000000000000000000000000000000000000000000800100008001800100000000000000000000000080010000000000000082009DFE1B
:3C972C0000800000000000000000000000000000000000000000000000000000000000000000000000000000000000000000000000000000000000D002006CFE45
:3C976800000000000000000000000000000000000000000000000000000000000000000000000000000000000000000000000000000000000000000002003CFE89
:3C97A400008006000000000000000000000000000000000000000000000000000000000000000000000000000000000000000000000000000000008006001EFE61
:3C97E00002800000000000000000000000000000000000000000000000000000000000000000000000000000000000000000000000000000000000800E0481FFB9
:3C981C0002D000000000000000000000000000000000000000000000000000000000000000000000000000000000000000000000000000000000008010006FFE41
:3C9858000000060000000000000000000000000000000000000000000000000000000000000000000000000000000000000000000000000000000000000078FE58
:3C989400020006000000000000000000000000000000000000000000000000000000000000000000000000000000000000000000010000000000008004009DFF6F
:3C98D0000200000000000000000000000000000000000000000000000000000000000000000000000000000000000000000000800000000000000000020115FFC3
:3C990C0000800000000000000000000000000000000000000000000000000000000000000000000000000000000000000000000000000000000000A20628E9FFE7
:3C9948000000000000000000000000000000000000000000000000000000000000000000000000000000000000000000000000000000000000000000060078FE67
:3C998400008006000000000000000000000000000000000000000000000000000000000000000000000000000000000000000000000000000000008002005AFE47
:3C99C00002800600000000000000000000000000000000000000000000000000000000000000000000000000000000000000000000000000000000800A10E3FE68
:3C99FC000280060000000000000000000000000000000000000000000000000000000000000000000000000000000000000000000000000000000080001049FED0
:3C9A38000000060000000000000000000000000000000000000000000000000000000000000000000000000000000000000000000000000000000000000069FF84
:3C9A7400020000000000000000000000000000000000000000000000000000000000000000000000000000000000000000000000000000000000008002008DFFA6
:3C9AB00002000000000000000000000000000000000000000000000000000000000000000000000000000000000000000000000000000000000000000C44F6FE34
:3C9AEC0000000000000000000000000000000000000000000000000000000000000000000000000000000000000000000000000000000000000000810600E8FFD0
:3C9B28000000000000000000000000000000000000000000000000000000000000000000000000000000000000000000000000000000000000000000060078FE85
:3C9B6400000000000000000000000000000000000000000000000000000000000000000000000000000000000000000000000000000000000000008000009EFEA9
:3C9BA00002000000000000000000000000000000000000000000000000000000000000000000000000000000000000000000000000000000000000A0080887FF51
:3C9BDC0002000000000000000000000000000000000000000000000000000000000000000000000000000000000000000000000000000000000000880000A7FF1D
:3C9C18000000008000800080008000800080008000800080008000800080008000800080008000800080008000800080008000800080008000800080060078FE14
:3C9C5400020000000000000000000000000000000000000000000000000000000000000000000000000000000000000000000000000000000000010000003FFF93
:3C9C90000200100100000000000000000000000000000000000000000000000000000000000000000000000000000000000000000000000000800020060061FE80
:3C9CCC00008000010000000000000000000000000000000000000000000000000000000000000000000000000000000000000000000000000000000000008EFE4F
:3C9D08000008000000000000000000000000000000000000000000000000000000000000000000000000000000000000000000000000000000000020000036FEC3
:3C9D4400000000000000000000000000000000000000000000000000000000000000000000000000000000000000000000000000000000000000000000001EFEC7
:3C9D8000000000000000000000000000000000000000000000000000000000000000000000000000000000000000000000000000000000000000000000001EFE8B
:3C9DBC00000000000000000000000000000000000000000000000000000000000000000000000000000000000000000000000000000000000000000000001EFE4F
:3C9DF800000000000000000000000000000000000000000000000000000000000000000000000000000000000000000000000000000000000000000000001EFE13
:3C9E3400000000000000000000000000000000000000000000000000000000000000000000000000000000000000000000000000000000000000000000001EFED6
:3C9E7000000000000000000000000000000000000000000000000000000000000000000000000000000000000000000000000000000000000000000000001EFE9A
:3C9EAC00000000000000000000000000000000000000000000000000000000000000000000000000000000000000000000000000000000000000022000001EFE3C
:3C9EE800008000000000000000000000000000000000000000000000000000000000000000000000000000000000000000000000000000000000000000009EFE22
:3C9F2400000000000000000000000000000000000000000000000000000000000000000000000000000000000000000000000000000000000000000000001EFEE5
:3C9F6000000000000000000000000000000000000000000000000000000000000000000000000000000000000000000000000000010000000000000010001EFF97
:3C9F9C00000000000000000000000000000000000000000000000000000000000000000000000000000000000000000000000000000000000000000000001EFE6D
:3C9FD800000000000000000000000000000000000000000000000000000000000000000000000000000000000000000000000000000000000000000000001EFE31
:3CA01400000000000000000000000000000000000000000000000000000000000000000000000000000000000000000000000000000000000000000000001EFEF4
:3CA05000000000000000000000000000000000000000000000000000000000000000000000000000000000000000000000000000000000000000000000001EFEB8
:3CA08C00000000000000000000000000000000000000000000000000000000000000000000000000000000000000000000000000000000000000000000001EFE7C
:3CA0C800000000000000000000000000000000000000000000000000000000000000000000000000000000000000000000000000000000000000000000001EFE40
:3CA10400000000000000000000000000000000000000000000000000000000000000000000000000000000000000000000000000000000000000000000001EFE03
:3CA14000000000000000000000000000000000000000000000000000000000000000000000000000000000000000000000000000000000000000000000001EFEC7
:3CA17C00000000000000000000000000000000000000000000000000000000000000000000000000000000000000000000000000000000000000000000001EFE8B
:3CA1B800000000000000000000000000000000000000000000000000000000000000000000000000000000000000000000000000000000000000000000001EFE4F
:3CA1F400000000000000000000000000000000000000000000000000000000000000000000000000000000000000000000000000000000000000000000001EFE13
:3CA23000000000000000000000000000000000000000000000000000000000000000000000000000000000000000000000000000000000000000000000001EFED6
:3CA26C00008000000000000000000000000000000000000000000000000000000000000000000000000000000000000000000000000000000000000000009EFE9A
:3CA2A8000000000000000000000000000000000000000000000000000000000000000000000000000000000000000000000000000800000000000000800096FE5E
:3CA2E400000000000000000000000000000000000000000000000000000000000000000000000000000000000000000000000000000000000000000000001EFE22
:3CA320000000000000000000000000000000000000000000000000000000000000000000000000000000000000000000000000002000000000000004000038FEA7
:3CA35C00000000000000000000000000000000000000000000000000000000000000000000000000000000000000000000000000000000000000000000001EFEA9
:3CA39800000000000000000000000000000000000000000000000000000000002000000000000000000000000000000000000000000000000000000000002FFF3B
:3CA3D4000080000000000000000000000000000000000000000000000000000000000000000000000000000000000000000000020000000000000024000098FE11
:3CA41000000000000000000000000000000000000000000000000000000000000000000000000000000000000000000000000000000000000000000000001EFEF4
:3CA44C00000080000000000000000000000000000000000000000000000000000000000020002000000000000000000000000000000000000000800000083CFE52
:3CA48800000000000000000000000000000000000000000000000000000000000000000000000000000000000000000000000000000000000000000000001EFE7C
:3CA4C4000020060000000000000000000000000000000000000000000000000000000000000000000000000000000000000000000000000000000000000058FEE0
:3CA500000000280000000000000000000000000000000000000000000000000000000000000000000000000000000000000000000000000000000002000096FE61
:3CA53C0000000000000000000000000000000000000000000000000000000000000000000080040000000000000000000000000000000080010000000048DFFEB9
:3CA57800000000000000000000000000000000000000000000000000000000000000000000000400000000000000000000000000000000000000000000001AFE8B
:3CA5B400000000000000000000000000000000000000000000000000000000000000000000800200000000000000000000000000000000800200000000001EFE4B
:3CA5F000020000000000000000000000000000000000000000000000000000000000000000804A00000000000000000000000000000000804A00000000002FFF6B
:3CA62C00020000000000000000000000000000000000000000000000000000000000000000800400000000000000000000000000000000800400000020200FFF9A
:3CA66800000000000000000000000000000000000000000000000000000000000000000000000200000000000000000000000000000000000200000000000FFFA4
:3CA6A400020000000000000000000000000000000000000000000000000000000000000000000200000000000000000000000000000000000200000000002FFF46
:3CA6E000020000000000000000000000000000000000000000000000000000000000000000004C00000000000000000000000000000000004C00000000003EFE68
:3CA71C0000000000000000000000000000000000000000000000000000000000000000000080020000000000000000000000000000000080010000820200ACFFCF
:3CA75800000000000000000000000000000000000000000000000000000000000000000000000200000000000000000000000000000000000000000002003EFE85
:3CA7940000000000000000000000000000000000000000000000000000000000000000000080020000000000000000000000000000000080020000800200BCFE49
:3CA7D000020000000000000000000000000000000000000000000000000000000000000000802A00000000000000000000000000000000802A0000A02A0027FF07
:3CA80C000200000000000000000000000000000000000000000000000000000000000000008002000000000000000000000000000000008004000080080021FF60
:3CA848000000000000000000000000000000000000000000000000000000000000000000000004000000000000000000000000000000000002000000000018FEB8
:3CA8840002000000000000000000000000000000000000000000000000000000000000000000020000000000000000000000000000000000020000800600C9FF44
:3CA8C000020000000000000000000000000000000000000000000000000000000000000000002C00000000000000000000000000000000002C000000860041FF3C
:3CA8FC0000000000000000000000000000000000000000000000000000000000000000000081000000000000000000000000000000000080090000A41600C4FE9A
:3CA938000000000000000000000000000000000000000000000000000000000000000000000000000000000000000000000000000000000000000000060078FE67
:3CA974000000000000000000000000000000000000000000000000000000000000000000000000000000000000000000000000000000008002000080000014FE93
:3CA9B000020000000000000000000000000000000000000000000000000000000000000000A0000000000000000000000000000000000080220000808600C1FF61
:3CA9EC00020000000000000000000000000000000000000000000000000000000000000040000600000000000000000000000000000000800C00008200002BFFAF
:3CAA2800000000000000000000000000000000000000000000000000000000000000000000000000000000000000000000000000000000000200000000001CFED6
:3CAA64000200000000000000000000000000000000000000000000000000000000000000008006000000000000000000000000000000000002000080000023FF8A
:3CAAA000020000000000000000000000000000000000000000000000000000000000000000200000000000000000000000000000000000002400002006006FFFA0
:3CAADC0000000000000000000000000000000000000000000000000000000000000000000000000000000000000000000000008015000080110000821648EFFE4B
:3CAB1800000000000000000000000000000000000000000000000000000000000000000000000000000000000000000000000000040000000000000000005EFEA1
:3CAB5400000000000000000000000000000000000000000000000000000000000000000000000000000000000000000000000080020000800200008006005AFEE3
:3CAB900002000000000000000000000000000000000000000000000000000000000000000000000000000000000000000000008022000080220000A020002DFF57
:3CABCC000200000000000000000000000000000000000000000000000000000000000000000000000000000000000000000000801400008014000088204035FE08
:3CAC0800000000000000000000000000000000000000000000000000000000000000000000000000000000000000000000000000020000000200000000002DFFE0
:3CAC440002000000000000000000000000000000000000000000000000000000000000000000000000000000000000000000000002000000020000800600EBFF5E
:3CAC8000020000000000000000000000000000000000000000000000000000000000000000000000000000000000000000000000240000002400002006003EFEEC
:3CACBC0002000000000000000000000000000000000000000000000000000000000000000081060000000000000000000000008001000080010000820600C4FF86
:3CACF800000000000000000000000000000000000000000000000000000000000000000000000000000000000000000000000000000000000000000000001EFE04
:3CAD3400000000000000000000000000000000000000000000000000000000000000000000000600000000000000000000000080020000800200008006005CFEF9
:3CAD7000000000000000000000000000000000000000000000000000000000000000000000A0000000000000000000000000008032000080320000A03000A7FF2D
:3CADAC0002000000000000000000000000000000000000000000000000000000000000004000000000000000000000000000008004000080040000A100005FFE23
:3CADE800020000000000000000000000000000000000000000000000000000000000000000000000000000000000000000000000020000000200000000001CFE0F
:3CAE24000000000000000000000000000000000000000000000000000000000000000000008000000000000000000000000000000200000002000080060043FFA6
:3CAE6000000000000000000000000000000000000000000000000000000000000000000000200000000000000000000000000000340000003400000006001DFE0D
:3CAE9C00020000000000000000000000000000000000000000000000000000000000000000000000000000000000000000000080010000800100009006489DFEFD
:3CAED8000000000000000000000000000000000000000000000000000000000000000000000000000000000000000000000000000000000000000000060078FEC2
:3CAF1400000000000000000000000000000000000000000000000000000000000000000000000000000000000000000000000080020000800200008000003CFE43
:3CAF5000000000000000000000000000000000000000000000000000000000000000000000000000000000000000000000000080920000808A0000A056007FFF35
:3CAF8C00020000000000000000000000000000000000000000000000000000000000000000000000000000000000000000000080040000800400008220006BFF73
:3CAFC800020000000000000000000000000000000000000000000000000000000000000000000000000000000000000000000000020000000200000000000DFF3B
:3CB0040000000000000000000000000000000000000000000000000000000000000000000000000000000000000000000000000002000000020000800000ADFFE0
:3CB04000000000000000000000000000000000000000000000000000000000000000000000000000000000000000000000000000940000008C00002006203EFF31
:3CB07C0002000000000000000000000000000000000000000000000000000000000000000000000000000000000000000000008001000080010000B01648ADFFDA
:3CB0B8000000000000000000000000000000000000000000000000000000000000000000000000000000000000000000000000000000000000000000060078FEE0
:3CB0F400000000000000000000000000000000000000000000000000000000000000000000000000000000000000000000000080020000800200008000003CFE62
:3CB13000000000000000000000000000000000000000000000000000000000000000000000000000000000000000000000000080120400800A040080060223FE16
:3CB16C000200000000000000000000000000000000000000000000000000000000000000000000000000000000000000000000800400008004000082001069FEA4
:3CB1A800020000000000000000000000000000000000000000000000000000000000000000000000000000000000000000000000020000000200000000000DFF59
:3CB1E40000000000000000000000000000000000000000000000000000000000000000000000000000000000000000000000000002000000020000800000ADFFFF
:3CB22000000000000000000000000000000000000000000000000000000000000000000000000000000000000000000000000000140400000C040020062076FF0F
:3CB25C0000000000000000000000000000000000000000000000000000000000000000000000000000000000000000000000008009000080110000820A48F3FED7
:3CB29800000000000000000000000000000000000000000000000000000000000000000000000000000000000000000000000000000000000000000002003CFE3E
:3CB2D400000000000000000000000000000000000000000000000000000000000000000000000000000000000000000000000080020000800200008002001EFE9C
:3CB3100002000000000000000000000000000000000000000000000000000000000000000000000000000000000000000000008002040080020100A002100BFF3A
:3CB34C000200000000000000000000000000000000000000000000000000000000000000000000000000000000000000000000800C0000801400008000087BFFA1
:3CB38800000000000000000000000000000000000000000000000000000000000000000000000000000000000000000000000000020000000200000000002DFF59
:3CB3C40002000000000000000000000000000000000000000000000000000000000000000000000000000000000000000000000002000000020000800600EBFFD7
:3CB4000002000000000000000000000000000000000000000000000000000000000000000000000000000000000000000000000004040000040100000E4494FF1C
:3CB43C000200000000000000000000000000000000000000000000000000408006000000008100000000000000000000000000800900008009000090064807FE96
:3CB478000000000000000000000000000000000000000000000000000000000006800000000000000000000000000000000000000000000000000000060076FE98
:3CB4B400000000000000000000000000000000000000000000000000000000000600000000000000000000000000000000000080020000800600008000003EFE92
:3CB4F000000000000000000000000000000000000000000000000000000000A00600000000A0000000000000000000000000008002020080860000C08E000BFFF8
:3CB52C000200000000000000000000000000000000000000000000000000000000000000400000000000000000000000000000800C000080060000820010EFFE10
:3CB56800020000000000000000000000000000000000000000000000000000000000000000000600000000000000000000000000020000000600000000000FFF89
:3CB5A40000000000000000000000000000000000000000000000000000000080000000000080000000000000000000000000000002000000000000800000AFFF3B
:3CB5E0000000000000000000000000000000000000000000000000000000000000800000002006000000000000000000000000000402000000000020064072FEAD
:3CB61C00000000000000000000000000000000000000000000000000000000000000000000000000000000000000000000000000100000001000008202487BFE8D
:3CB65800000000000000000000000000000000000000000000000000000000000000000000000000000000000000000000000000000000000000000002003CFE7A
:3CB6940000000000000000000000000000000000000000000000000000000000000000000000000000000000000000000000000000000000000000800200BCFE3E
:3CB6D00002000000000000000000000000000000000000000000000000000000000000000000000000000000000000000000000000020000000200A00A0885FF02
:3CB70C000200000000000000000000000000000000000000000000000000000000000000000200000000000000000000000080000000800000000080005043FEEC
:3CB748000080008000800080008000800080008000800080008000800080008000800080008000800080008000800080008000800080000000800080000007FF3F
:3CB784000200000000000000000000000000000000000000000000000000000000000000000000000000000000000000000000000000000000000000060049FF39
:3CB7C00002000000000000000000000000000000000000000000000000000000000000000040000000000000000000000000004000000040000000000E01C4FEBA
:3CB7FC000000000000000000000000000000000000000000000000000000000000000000004201000000000000000000000000020100000201000000000068FE62
:3CB83800000000000000000000000000000000000000000000000000000000000000000000200000000000000000000000000008080100080801002000008CFEE8
:3CB87400000000000000000000000000000000000000000000000000000000000000000000000000000000000000000000000000000000000000000000001EFE7C
:3CB8B000000000000000000000000000000000000000000000000000000000000000000000000000000000000000000000000000000000000000000000001EFE40
:3CB8EC00000000000000000000000000000000000000000000000000000000000000000000000000000000000000000000000000000000000000000000001EFE04
:3CB928000000000000000000000000000000000000000000000000000000000000000000000000000000000000000000000000000000000002000000080094FE47
:3CB96400000000000000000000000000000000000000000000000000000000000000000000000000000000000000000000000000000000000000000000001EFE8B
:3CB9A00000000000000000000000000000000000000000000000000000000000000004000008000000000000000000000000000000000000000000000000DEFE83
:3CB9DC000000000000000000000000000000000000000000000000000000000000000000000000000000000000000000000000000000008000000000200094FEFD
:3CBA18000000000000000000000000000000000000000000000000000000000000000000000000000000000000000000000000800000000000000000000016FE5E
:3CBA5400000000000000000000000000000000000000000000000000000000000000000000000400000000000000000000000000000400000004000000005AFE52
:3CBA9000000000000000000000000000000000000000000000000000000000000000000000000000000000000000000000000000000000000000000000001EFE5E
:3CBACC00000000000000000000000000000000000000000000000000000000000000000000000000000000000000000000000000000000000000000000001EFE22
:3CBB080002000000000000000000000000000000000000000000000000000800000000000000000000000000000000000000000000000000000000000000B6FE43
:3CBB440000000000000000000000000000000000000000000000000000000000000000000000000000000000000000000000000009000000410000004000DAFF62
:3CBB80000000000000000000000000000000000000000000000000000000000000000000000000000000000000000000000000800040000000000000000056FE75
:3CBBBC0000000000000000000000000000000000000000000000000000000000000000000800400000000000000000000000000000000000000000000000D6FE31
:3CBBF800000000000000000000000000000000000000000000000000000000000000000000000000000000000000000000000000000000000000000000001EFEF5
:3CBC3400000000000000000000000000000000000000000000000000000000000000000000000000000000000000000000000000000000000000000000001EFEB8
:3CBC7000000000000000000000000000000000000000000000000000000000000000000000000000000000000000000000000000000000006000000050006AFF7F
:3CBCAC00000000000000000000000000000000000000000000000000000000000000000000000000000000000000000000000000000000000000000000001EFE40
:3CBCE800000000000000000000000000000000000000000000000000000000000000000000000000000000000000000000000000000000000000000000001EFE04
:3CBD2400000000000000000000000000000000000000000000000000000000000000000000000000000000000000000000000000000000000000000000001EFEC7
:3CBD6000000000000000000000000000000000000000000000000000000000000000000000000000000000000000000000000000000000000000000000001EFE8B
:3CBD9C000000000000000000000000000000000000000000000000000000000000000000000000000000000000000000000000800000000000000000000016FED7
:3CBDD80000000000000000000000000000000000000000000000000000000000000000000000000000000000000000000000000000000000880000000004D6FECF
:3CBE1400000000000000000000000000000000000000000000000000000000000000000000000000000000000000000000000000000000000000000000001EFED6
:3CBE5000000000000000000000000000000000000000000000000000000000000000000000000000000000000000000000000040001000000000000000000AFE5E
:3CBE8C000000000000000000000000000000000000000000000000000000001000000000000000000000000000000000000000000000000000000100018086FE64
:3CBEC800000000000000000000000000000000000000000000000000000000000000000000100000000000000000000000000000000000000000000200001CFF11
:3CBF0400000000000000000000000000000000000000000000000000000000000000000000000000000000000000000000000000000000000000000000001EFEE5
:3CBF40000000000000000000000000000000000000000000000000000000000000000000000000000000000000000000000000100004001020000000200028FE3B
:3CBF7C0000000000000000000000000000000000000000000000000000000000000000000000000000000000000000000000000000000000201000000008AEFFA4
:3CBFB80000000000000000000000000000000000000000000000000000000000000000000000080000000000000000000000200000002000080080000000B4FECB
:3CBFF400000000000000000000000000000000000000000000000000000000080000000000080000000000000000000000000028060000000000004008003CFE51
:3CC030000000000000000000000000000000000000000000000000000000000000000000800000010000000000000000000000000000000000010020000036FEFE
:3CC06C0000000000000000000000000000000000000000000000000000000000000000000000000000000000048000000000000000000000004800480000D6FEB0
:3CC0A8000000000000000000000000000000000000000000000000000000000000000000000000800480000000000400048000000000000000800000000052FE00
:3CC0E40000000400040004800000008000800480040000000480040000000000000000000000048004800000048004000480040000000000008000800000D6FE98
:3CC12000000000800080000004800400040000000080048000000080048004800480048004800000000004800000008000000080048004800480048000005EFE4F
:3CC15C0000000480048004800480048004800480048004800480048004800480048004800480048004800480048004800480048004800480048104B000002EFF5D
:3CC1980000000400040004800000008000800480040000000480040000000000000000000000048004800000048004000480040000000000008000800000D6FEE3
:3CC1D400000000800080000004800400040000000080048000000080048004800480048004800000000004800000008000000080048004800480048000005EFE9B
:3CC2100000000080008000000480040004000000008004800000008004800480048004800480000000000480000000800000008004800480044004000000D2FEAA
:02C24C00FFFFF2
:00000001FF
